:0200000480007A
:10000000B72F0000938F0F8073900F306F00400365
:100010001300000013000000130000001300000094
:100020001300000013000000130000001300000084
:100030001300000013000000130000001300000074
:100040009702000093824211739052309300000097
:10005000130100009301000013020000930200004E
:100060001303000093030000130400009304000036
:10007000130500009305000013060000930600001E
:100080001307000093070000130800009308000006
:100090001309000093090000130A0000930A0000EE
:1000A000130B0000930B0000130C0000930C0000D6
:1000B000130D0000930D0000130E0000930E0000BE
:1000C000130F0000930F000097110200938181CD60
:1000D000170502001305054F979503009385457D8D
:1000E00013060000EF00001A1705020013058542F1
:1000F000970502009385C54A13060000EF0080189B
:1001000017A503001305057B97B503009385457A72
:1001100037B6ABAB1306B6BAEF00C01617B1030083
:1001200013014179EF80D0689392120093D21200AC
:100130009382D2FF638A02008322010013014100EF
:100140006F0000177300203083220100130141006B
:10015000730020301301C1FF23205100F32220340B
:10016000E3C402FC8322010013014100130141F8A2
:1001700023221100232421002326310023284100BB
:10018000232A5100232C6100232E71002320810299
:10019000232291022324A1022326B1022328C10293
:1001A000232AD102232CE102232EF1022320010570
:1001B0002322110523242105232631052328410567
:1001C000232A5105232C6105232E71052320810745
:1001D000232291072324A1072326B1072328C1073F
:1001E000232AD107232CE107232EF107732520347E
:1001F000F3251034130601006F000000731015344E
:1002000083204100032181008321C10003220101D9
:1002100083224101032381018323C10103240102BD
:1002200083244102032581028325C10203260103A1
:1002300083264103032781038327C1030328010485
:1002400083284104032981048329C104032A010569
:10025000832A4105032B8105832BC105032C01064D
:10026000832C4106032D8106832DC106032E010731
:10027000832E4107032F8107832FC1071301C10775
:10028000730020302320C5006376B50013054500B8
:100290006FF05FFF678000000000000000000000BA
:1002A000000000000000000000000000000000004E
:1002B000130101F8232011002322210023243100FF
:1002C0002326410023285100232A6100232C71009A
:1002D000232E8100232091022322A1022324B10294
:1002E0002326C1022328D102232AE102232CF10272
:1002F000232E010323201105232221052324310568
:100300002326410523285105232A6105232C710545
:10031000232E8105232091072322A1072324B1073F
:100320002326C1072328D107232AE107232CF1071D
:100330009702020083A2022323A02200F32210349A
:10034000232E5106EF00C03B17010200032181213B
:10035000032101008322C10773901234B7220000E9
:100360009382028873A00230832001000322C1001F
:100370008322010103234101832381010324C1015D
:100380008324010203254102832581020326C10241
:100390008326010303274103832781030328C10325
:1003A000832801040329410483298104032AC10409
:1003B000832A0105032B4105832B8105032CC105ED
:1003C000832C0106032D4106832D8106032EC106D1
:1003D000832E0107032F4107832F81071301010893
:1003E00073002030970202009382C21D23A01200E6
:1003F00023A2220023A4320023A6420023A85200F5
:1004000023AA620023AC720023AE820023A09202D2
:1004100023A2A20223A4B20223A6C20223A8D202CC
:1004200023AAE20223ACF20223AE020323A01205A8
:1004300023A2220523A4320523A6420523A85205A0
:1004400023AA620523AC720523AE820523A092077E
:1004500023A2A20723A4B20723A6C20723A8D20778
:1004600023AAE20723ACF207EF70803417010200E1
:100470000321410F032101008322C107739012342D
:10048000B72200009382028873A00230832001000B
:100490000322C1008322010103234101832381013F
:1004A0000324C10183240102032541028325810223
:1004B0000326C10283260103032741038327810307
:1004C0000328C103832801040329410483298104EB
:1004D000032AC104832A0105032B4105832B8105CF
:1004E000032CC105832C0106032D4106832D8106B3
:1004F000032EC106832E0107032F4107832F810797
:100500001301010873002030970202009382820BCE
:1005100083A0020003A1420083A1820003A2C200C3
:1005200083A2020103A3420183A3820103A4C201A7
:1005300083A4020203A5420283A5820203A6C2028B
:1005400083A6020303A7420383A7820303A8C2036F
:1005500083A8020403A9420483A9820403AAC20453
:1005600083AA020503AB420583AB820503ACC20537
:1005700083AC020603AD420683AD820603AEC2061B
:1005800083AE020703AFC20983AF82076780000012
:1005900073700430130101F823201100232221007D
:1005A000232431002326410023285100232A6100FF
:1005B000232C7100232E8100232091022322A102EB
:1005C0002324B1022326C1022328D102232AE102D7
:1005D000232CF102232E01032320110523222105C0
:1005E000232431052326410523285105232A6105AB
:1005F000232C7105232E8105232091072322A10797
:100600002324B1072326C1072328D107232AE10782
:10061000232CF1079702020083A2C2F423A0220038
:10062000232E1106EF30103517010200032181F34C
:10063000032101008322C10773901234B722000006
:100640009382028873A00230832001000322C1003C
:100650008322010103234101832381010324C1017A
:100660008324010203254102832581020326C1025E
:100670008326010303274103832781030328C10342
:10068000832801040329410483298104032AC10426
:10069000832A0105032B4105832B8105032CC1050A
:1006A000832C0106032D4106832D8106032EC106EE
:1006B000832E0107032F4107832F810713010108B0
:1006C00073002030737004306F00000073104530E9
:1006D000678000007325403073F04330678000006E
:1006E00097070000938747FE232EB5FE2322C5FA05
:1006F000232635F82320F5F8130505F86780000058
:10070000130101FF23261100EF704007EF20505D19
:10071000631805008320C1001301010167800000F8
:100720008320C100130101016F30D024130101FEA9
:10073000232631019309050013058003232A910024
:1007400023244101232E1100232C81002328210181
:100750002322510193840500130A0600EF50D03D77
:1007600063040512970702009387C7DB83A707007E
:10077000130405006388070A639C040813094400F6
:100780001305090023269402231A04022328440394
:1007900023203401EF00005213058401EF00805143
:1007A000970702009387C7D703A707000325C40252
:1007B00093072000B38497402328840023228402D7
:1007C000232C9400636AA70493172500B387A7001E
:1007D0009397270017050200130585E63305F500FA
:1007E00093050900EF00804D130510008320C1011F
:1007F0000324810183244101032901018329C100CC
:10080000032A8100832A410013010102678000004E
:10081000930410006FF09FF69707020023A2A7D061
:100820006FF09FFA17050200130585E19707020094
:1008300023AA87CEEF00004617050200130585E1C5
:10084000EF004045970A0200938A0AE213850A00E6
:10085000EF00404417090200130949E2130509009B
:10086000EF00404317050200130585E2EF008042C8
:100870009707020023AC57CB9707020023A627CB8C
:10088000E38E04EE6FF0DFF81305F0FF6FF01FF654
:10089000130101FE232A910023282101970402005D
:1008A000938444C817090200130949C783A70400A9
:1008B000232C81000324090023263101232E11005B
:1008C000330485001385470093890500EF004047F6
:1008D00083A504008327090023A285006372F40422
:1008E00097070200938747C403A507009385450037
:1008F000EF00C03F6382090483A504000324810143
:100900008320C101832441010329010113850900CA
:100910008329C10093858501130101026F00003D09
:1009200097070200938787C003A5070093854500BA
:10093000EF00C03BE39209FC8320C1010324810145
:1009400083244101032901018329C100130101020C
:1009500067800000130101FD23202103232E3101B4
:10096000232611022324810223229102232C4101F8
:10097000232A51012328610123267101170902004E
:10098000130909CC8327090597090200938949B9FE
:1009900063800706737004308327C90503A4C7006A
:1009A00013058401EF00C0397360043093044400E0
:1009B00013850400EF00C0388327C40283A6090012
:1009C00093850400139527003305F50013152500C2
:1009D000130705003305A90063F2F61C1707020090
:1009E0002320F7B4EF00802D83270905E39407FA4D
:1009F000EF20902297070200938707B203A7070012
:100A0000970A0200938A8AB183A70A003305E5405A
:100A1000170702002320A7B0170A0200130A0AB121
:100A2000970B0200938B4BB0170B0200130B8BAE8E
:100A3000630A050C938717001305F5FF17070200DB
:100A4000232EF7AC170702002326A7AC03270A00C2
:100A5000639E070083A60B00170602002326E6AC60
:100A6000170702002324D7AC13870600832607004C
:100A7000E38006FC0327C7000324C70003274400C4
:100A800063FEE7006FF0DFFA03A7C70083A70A0041
:100A90000324C7000327440063E2E70673700430B1
:100AA0009304440013850400EF0080298327840207
:100AB0001305840163840700EF008028736004300D
:100AC0008327C40203A70900938504001395270018
:100AD0003305F500131525003305A9006376F700EB
:100AE00017070200232EF7A2EF00401D83270A00FC
:100AF00003A70700E31A07F883A70A0003250B00E2
:100B0000E31A05F283A60900170702002326F7A0BF
:100B1000939726003387D700131727003307E90080
:100B200003270700631E0708638406049387F6FF04
:100B3000139727003307F700131727003307E9003F
:100B40000327070063160706638007029387E6FF03
:100B5000139727003307F700131727003307E9001F
:100B6000032707006316070417070200232AF79AD2
:100B70008320C1020324810283244102032901024C
:100B80008329C101032A8101832A4101032B010129
:100B9000832BC10013010103678000003305E900C6
:100BA000EF00C01183270905E39607DE6FF05FE4CD
:100BB00093860700170702002324F79693972700D0
:100BC000B387D700939727003307F90083264700A0
:100BD000938787003309F90083A746002322F70093
:100BE0006382270503A5C700032481028320C10275
:100BF0009707020023A8A792832441020329010238
:100C00008329C101032A8101832A4101032B0101A8
:100C1000832BC10003230500832505031301010372
:100C20006700030083A747002322F7006FF09FFBB4
:100C3000130101FF232611002322910023248100A8
:100C40008327C50003A4C70093048401138504000F
:100C5000EF00000F9385040017050200130545A35C
:100C6000EF00C005970702009387C78B83A7070093
:100C70000325C4028320C10083A7C7020324810087
:100C8000832441003335F50013451500130101019C
:100C900067800000930785001307F0FF2322F5000B
:100CA0002324E5002326F5002328F5002320050052
:100CB0006780000023280500678000008327450027
:100CC00023A2F50003A7870023A4E50003A787005C
:100CD0002322B70023A4B70023A8A500832705007B
:100CE000938717002320F5006780000003A6050006
:100CF0009307F0FF130785006316F6006F0080036B
:100D0000138707008327470083A60700E37AD6FEF0
:100D100023A2F50023A4B70023A4E5002322B700F3
:100D200023A8A50083270500938717002320F5003B
:100D30006780000003270501832747006FF05FFDF0
:100D40000327450083268500832705012324D70038
:100D500003278500832645002322D70003A74700E9
:100D60006316A7000327850023A2E70023280500B8
:100D700003A507001305F5FF23A0A7006780000067
:100D80000326050493870500630406028325C50036
:100D900003274500B385C5002326B50063E6E500BB
:100DA000832505002326B500138507006F50407981
:100DB00067800000130101FF232481002326110016
:100DC0001304050023229100EF30106F8327840461
:100DD000635AF004832744026386070493044402A1
:100DE0006F000002832784049387F7FF2324F40411
:100DF000832784046358F002832744026384070234
:100E000013850400EF30501AE30E05FCEF30104755
:100E1000832784049387F7FF2324F404832784041F
:100E2000E34CF0FC9307F0FF2324F404EF30106C44
:100E3000EF30906883274404635AF0048327040149
:100E400063860704930404016F00000283274404AF
:100E50009387F7FF2322F404832744046358F002A6
:100E6000832704016384070213850400EF30D01345
:100E7000E30E05FCEF309040832744049387F7FF8F
:100E80002322F40483274404E34CF0FC9307F0FF8F
:100E90002322F404032481008320C1008324410021
:100EA000130101016F309064630A0508130101FE0C
:100EB000232C810013040500232E1100232A910006
:100EC000232821012326310113890500EF30D05E4C
:100ED000832404048325C4038329040013850400A8
:100EE000EF7050671307F0FF232C0402B3079540FF
:100EF000B387F9003385A9002322E4042322A40048
:100F0000232434012326F4002324E404631C09026F
:100F10008327040163920704EF30505D8320C101F1
:100F20000324810183244101032901018329C10094
:100F30001305100013010102678000007370043074
:100F40006F00000013050401EFF0DFD41305440225
:100F5000EFF05FD46FF05FFC13050401EF30D004B5
:100F600093071000E31AF5FAEFF08FE26FF0DFFA63
:100F700063160500737004306F000000130101FE5A
:100F8000232A91002328210123263101232E110039
:100F9000232C8100930405001389050093090600A2
:100FA0006380050AEF70105B13055505EF50C038DC
:100FB00013040500630E0508930745052320F5007B
:100FC000232E940223202405EF30104F83240404A1
:100FD0008325C4030329040013850400EF70905790
:100FE0009306F0FF232C0402B30795403307A900B2
:100FF000B307F9002322D4042322E4002326F400BB
:101000002324D4041305040123242401EFF09FC8F2
:1010100013054402EFF01FC8EF30504D230834058C
:10102000130504008320C1010324810183244101AD
:10103000032901018329C100130101026780000017
:1010400013054005EF50402F1304050063160500FB
:10105000737004306F000000232084006FF05FF68F
:1010600063160500737004306F0000006376B500EE
:10107000737004306F000000130101FF232481000E
:101080001306200013840500930500002326110099
:10109000EFF01FEE630C0500232C85028320C100B6
:1010A0000324810013010101678000007370043084
:1010B0006F000000130101FB232611042324810487
:1010C0002322910423202105232E3103232C4103C5
:1010D000232A510323286103232671032326C100F9
:1010E00063060528638C052693072000639CF600A1
:1010F0000327C503930710006306F70073700430DD
:101100006F00000013890600938405001304050096
:10111000EF30D01A631A05008327C10063860700E9
:10112000737004306F000000EF3010390327840320
:101130008327C403130B0000930B20009309F0FFD7
:10114000130A0401930A44026364F71063047923C9
:101150008327C1006382073663160B0013058101E4
:10116000EF30407FEF309038EF208029EF30D034DF
:1011700083274404639437012322040483278404CF
:101180006394370123240404EF3050369305C100E3
:1011900013058101EF30007F63160530EF30D03149
:1011A000032784038327C4036304F710EF3010344C
:1011B000EF309030832784046346F0026F00000311
:1011C00013850A00EF30405E63040500EF30100B1A
:1011D000832784049387F7FF2324F404832784045C
:1011E0006356F00083274402E39C07FC2324340564
:1011F000EF30D02FEF30502C832744046346F002A9
:101200006F00000313050A00EF30005A6304050065
:10121000EF30D006832744049387F7FF2322F4049A
:10122000832744046356F00083270401E39C07FCF2
:1012300023223405EF30902BEF200050130B1000C9
:10124000EF309027032784038327C403E370F7F06C
:101250000326040463040612631A091E032584008E
:1012600093850400EF50C02D832784008326040457
:1012700003274400B387D7002324F40063E4E71076
:1012800083278403832604000327440293871700DF
:101290002324D400232CF402630007101305440216
:1012A000EF308050930710006318F50E6F00401464
:1012B000EF30D0238325C10013050A00EF30C02191
:1012C000EF30901F832784046346F0026F00000311
:1012D00013850A00EF30404D63040500EF30007ABB
:1012E000832784049387F7FF2324F404832784044B
:1012F0006356F00083274402E39C07FC2324340553
:10130000EF30D01EEF30501B832744046346F002B9
:101310006F00000313050A00EF3000496304050065
:10132000EF30C075832744049387F7FF2322F4042A
:10133000832744046356F00083270401E39C07FCE1
:1013400023223405EF30901AEF20003FE31805EE1A
:10135000EFF00FA4130B10006FF09FEE832705042E
:10136000E38407D8737004306F000000737004309A
:101370006F0000000326040463100608832704009E
:101380006386070483278403032744029387170097
:10139000232CF402E31407F0EF305015130510006E
:1013A0008320C1040324810483244104032901040C
:1013B0008329C103032A8103832A4103032B0103E9
:1013C000832BC1021301010567800000032544003F
:1013D000EF30900183278403032744022322040073
:1013E00093871700232CF402E31A07EAE30605FAB1
:1013F000EFF00F9A6FF05FFA0325C40093850400A5
:10140000EF500014832704040327C400832604003C
:10141000B307F0403307F7002326E400637ED704C8
:1014200003274400B307F7002326F4001307200026
:10143000832744026304E904032784031307170086
:10144000232CE402E38A07F46FF05FE50325C40070
:1014500093850400EF50C00E832704040327C400C3
:1014600083260400B307F0403307F7002326E40087
:10147000E37ED7FA6FF0DFFA832744020327840361
:10148000E30C07FA032784031307F7FF232CE40276
:101490000327840313071700232CE402E38E07EECF
:1014A0006FF0DFDF13050400EFF0DF90EF20C028BE
:1014B000130500006FF0DFEEEF305003130500005E
:1014C0006FF01FEE130101FF23229100930405002A
:1014D000130540052324810023261100EF40D06529
:1014E00013040500630C0504232C05029307F0FF89
:1014F0002322F5041307100013050501232EE4022F
:101500002324F404232204002320040023240400C1
:10151000232604002320040423089404EFF08FF70B
:1015200013054402EFF00FF79306000013060000C6
:101530009305000013050400EFF0DFB71305040066
:101540008320C10003248100832441001301010191
:101550006780000063040504130101FF2324810058
:101560002322910023261100232021010329450075
:1015700013040500EF308053930400006304A902B4
:101580008320C10003248100138504000329010086
:10159000832441001301010167800000737004304F
:1015A0006F0000008327C400930410009387F7FFA7
:1015B0002326F400E39607FC9306000013060000C0
:1015C0009305000013050400EFF0DFAE6FF05FFB42
:1015D0006302050A63880508130101FE232C8100BC
:1015E000232A91002328210123244101232E1100C5
:1015F0002326310193072000938406001309060077
:10160000138A050013040500639CF6000327C50335
:10161000930710006302F70A737004306F00000034
:10162000EFF04F8B032784038327C403930905003E
:101630006366F7049304000013850900EFF00F8937
:101640008320C101032481011385040003290101C2
:10165000832441018329C100032A8100130101026F
:101660006780000083270504E38807F67370043061
:101670006F000000737004306F0000000326040444
:10168000631E060C832704006386071283278403E6
:101690001307F0FF93871700232CF4028327840499
:1016A0006388E70E83278404930410009387170050
:1016B0002324F4046FF05FF8EFF0CF810327840355
:1016C0008327C403930905006360F7060326040417
:1016D000E30A06FA0325C40093050A00EF405066AA
:1016E000832704040327C40083260400B307F040C3
:1016F0003307F7002326E4006378D700032744006C
:10170000B307F7002326F40093072000E390F4F8D2
:1017100083278403E38C07F6832784039387F7FFEB
:10172000232CF4026FF09FF603260404E30C06F466
:101730000325C40093050A00EF409060832704044A
:101740000327C40083260400B307F0403307F700E3
:101750002326E400E364D7FA6FF09FFBE39C04F6D2
:101760000325840093050A00EF40905D83278400E1
:101770008326040403274400B387D7002324F400FE
:10178000E3E6E7F0832704002324F4006FF01FF062
:101790008327440293041000E38007EA1305440200
:1017A000EF308000E30A05E8E30809E82320990008
:1017B0006FF09FE803254400EF300043232204002C
:1017C0006FF0DFEC6302050A8327050463860700D8
:1017D000737004306F00000083270500638A0708D8
:1017E000130101FE232C8100232A9100130405001C
:1017F0002328210123263101232E110013890500FE
:10180000EFE05FED032784038327C40393090500FA
:10181000930400006376F702832784031307F0FF25
:1018200093871700232CF40283278404638AE70438
:101830008327840493041000938717002324F4045F
:1018400013850900EFE09FE88320C1010324810193
:101850001385040003290101832441018329C10068
:101860001301010267800000737004306F000000F4
:1018700083274500E38607F6737004306F0000008D
:101880008327440263960700930410006FF05FFB08
:1018900013054402EF205071E30805FEE30609FE3C
:1018A000930710002320F9006FF01FFE130101FCC5
:1018B000232E1102232C8102232A910223282103A3
:1018C0002326310323244103232251032326C1006D
:1018D00063060528638C0526938A06009389050014
:1018E00013040500EF30801D631A05008327C10033
:1018F00063860700737004306F000000EF30C03B58
:10190000832784036394071C8327C1006380071027
:1019100013058101EF3000049304F0FF1309440222
:10192000130A0401EF30803CEF10902DEF30C038E7
:1019300083274404639497002322040483278404A8
:101940006394970023240404EF30403A9305C100C8
:1019500013058101EF30000363100524EF30C0351B
:1019600083278403638A070AEF304038EF30C0349E
:10197000832784046346F0026F0000031305090007
:10198000EF20906263040500EF30400F832784044A
:101990009387F7FF2324F404832784046356F0001D
:1019A00083274402E39C07FC23249404EF30003493
:1019B000EF308030832744046346F0026F00000359
:1019C00013050A00EF20505E63040500EF30000BA2
:1019D000832744049387F7FF2322F40483274404D6
:1019E0006356F00083270401E39C07FC2322940440
:1019F000EF30C02FEF105054EF30002C83278403BA
:101A00006396070C8327C100E39E07F0EF30002E9A
:101A1000130500006F00800FEF30402D8327040076
:101A2000638807108325C10013050900EF20D02A21
:101A3000EF308028832784046346F0026F000003A0
:101A400013050900EF20505663040500EF30000332
:101A5000832784049387F7FF2324F40483278404D3
:101A60006356F00083274402E39C07FC232494047C
:101A7000EF30C027EF304024832744046346F00250
:101A80006F00000313050A00EF20105263040500E5
:101A9000EF20D07E832744049387F7FF2322F404AA
:101AA000832744046356F00083270401E39C07FC6A
:101AB00023229404EF308023EF10104863040508BC
:101AC000EF30801F83278403E38E07F2938509009C
:101AD000130504008324C400EFF08FAA63940A085E
:101AE00083278403032704009387F7FF232CF40242
:101AF00063160700EF30C0262322A40083270401C9
:101B000063920708EF30801E130510008320C10385
:101B10000324810383244103032901038329C10290
:101B2000032A8102832A4102130101046780000015
:101B3000EF30801803254400EF20107BEF30001BAE
:101B40006FF05FEEEFE0DFA46FF09FF783270504EF
:101B5000E38407D8737004306F00000073700430A2
:101B60006F0000008327440223269400E38C07F8CB
:101B700013054402EF205043E30605F8EFE05FA1B0
:101B80006FF05FF813050401EF2010429307100077
:101B9000E31AF5F66FF09FFE13050400EFF08FA136
:101BA000EF109039130500006FF05FF66300050633
:101BB000130101FF2324810023202101232611008A
:101BC0002322910083244500138905001304050096
:101BD000EF20D06D6380A404930600001306090073
:101BE0009305000013050400EFF05FCC930710008D
:101BF000630CF5028320C10003248100832441008B
:101C00000329010013010101678000007370043093
:101C10006F0000008327C40013051000938717008E
:101C20002326F4006FF01FFD8327C400938717005D
:101C30002326F4006FF01FFC630805066386050C7D
:101C4000130101FE232C8100232A91002328210166
:101C5000232631012324410113040500232E110002
:101C60001309060093890500EFE0DFA683278403AC
:101C7000130A050093040000639C070213050A0081
:101C8000EFE0DFA48320C101032481011385040058
:101C900003290101832441018329C100032A810012
:101CA0001301010267800000737004306F000000B0
:101CB00003260404630406028325C400832744002A
:101CC000B385C5002326B40063E6F5008325040030
:101CD0002326B40013850900EF4090068327840370
:101CE0001307F0FF9387F7FF232CF40283274404A4
:101CF0006384E7028327440493041000938717004A
:101D00002322F4046FF09FF783270504E38A07F288
:101D1000737004306F00000083270401639607008E
:101D2000930410006FF09FF513050401EF20D027F6
:101D3000E30805FEE30609FE930710002320F900DF
:101D40006FF01FFE6306050883270504638A0508F4
:101D500063840708130101FE232C8100232A9100CC
:101D6000232821012324410113040500232E1100FF
:101D700023263101138A0500EFE0DF9583278403D2
:101D80001309050093040000638E07008329C40033
:101D900093050A0013050400EFE09FFE9304100072
:101DA0002326340113050900EFE05F928320C1016F
:101DB00003248101138504000329010183244101C7
:101DC0008329C100032A81001301010267800000FA
:101DD000737004306F000000737004306F000000F7
:101DE000E38C07FE737004306F000000631605007B
:101DF000737004306F000000130101FF2324810081
:101E00001304050023261100EF20106B0324840324
:101E1000EF20D06D8320C10013050400032481004E
:101E20001301010167800000631605007370043020
:101E30006F000000130101FF2326110023248100FD
:101E400013040500EF205067832784030324C40391
:101E50003304F440EF209069130504008320C1008F
:101E6000032481001301010167800000630605005F
:101E70000325850367800000737004306F00000045
:101E800063080504978703009387C79E03A747004D
:101E90006304E50403A7C7006302E50803A747013D
:101EA000630AE50603A7C7016302E50603A7470225
:101EB000630AE50403A7C7026302E50403A7470317
:101EC000630AE50203A7C7036302E5026F40C05E31
:101ED000737004306F000000130700001317370001
:101EE000B387E70023A007006F40005D1307700071
:101EF0006FF0DFFE130760006FF05FFE1307500006
:101F00006FF0DFFD130740006FF05FFD1307300037
:101F10006FF0DFFC130720006FF05FFC1307100069
:101F20006FF0DFFB0325C504678000002326B5049E
:101F30006780000003450505678000006308050011
:101F40000325850313351500678000007370043086
:101F50006F000000630C0500832785030325C5037C
:101F60003305F540133515006780000073700430A9
:101F70006F000000130101FF232481002322910040
:101F800023202101232611001304050013890500D5
:101F90009304060073700430EF201052032784036B
:101FA0008327C4036306F708EF205054736004309E
:101FB00073700430032784038327C40313050000D0
:101FC0006360F702736004308320C1000324810042
:101FD00083244100032901001301010167800000EF
:101FE00003260404630A06060325840093050900FA
:101FF000EF40005583278400832604040327440010
:10200000B387D7002324F40063E6E70083270400A6
:102010002324F400832784030327440293871700B3
:10202000232CF40263160704130510006FF09FF9C8
:10203000EF20D04B63980404736004308320C10008
:1020400003248100832441000329010013050000BB
:10205000130101016780000083270400E39C07FA55
:1020600003254400EF205038232204006FF09FFA2C
:1020700013054402EFE0DFBBE30805FA1305B0FFE8
:102080006FF05FF49305040113850400EFE05F80B7
:10209000736004301305C0FF6FF01FF3130101FFDD
:1020A00023248100232611001304050073700430DB
:1020B00083278503639007026310060A7360043068
:1020C0008320C100032481001305000013010101D6
:1020D00067800000736004307370043083278503C9
:1020E00013050000639C0700736004308320C10067
:1020F000032481001301010167800000138705009C
:10210000032604048325C40083274400B385C50047
:102110002326B40063E6F500832504002326B400DB
:1021200083278403130507009387F7FF232CF4020A
:10213000EF40004183270401639607001305100058
:102140006FF09FFA13050401EFE09FAEE30805FE70
:102150001305B0FF6FF05FF9930545021305060004
:10216000EFE00FF3736004301305C0FF6FF01FF84A
:10217000130101FF23229100232611002324810053
:10218000032785038327C50393040600636EF700C6
:102190008320C100032481001385040083244100AF
:1021A00013010101678000000326050413040500E4
:1021B000630A060403258500EF40803883278400E6
:1021C0008326040403274400B387D7002324F400A4
:1021D00063E6E700832704002324F40083278403B5
:1021E00093871700232CF402E39404FA8327440214
:1021F000E38007FA13054402EFE09FA3B334A00085
:102200006FF01FF983270500E39A07FC03254500BB
:10221000EF20901D232204006FF05FFC83278503CD
:1022200063820708130101FF232611002324810084
:10223000232291008327C5000328050403274500B6
:10224000B38707012326F50063E6E700832705002F
:102250002326F50083268503138705009385070051
:102260009387F6FF232CF502930406001304050060
:102270001306080013050700EF40802C83A7040015
:102280006396070083270401639207028320C1003D
:102290000324810083244100130510001301010170
:1022A000678000001305000067800000130504012B
:1022B000EFE01F98E30C05FC9307100023A0F40047
:1022C0006FF0DFFC977703009387C75A03A70700D7
:1022D0006300070403A787006308070403A7070137
:1022E0006308070403A787016308070403A707021D
:1022F0006308070403A787026308070403A707030B
:10230000630C070403A787036304070467800000C6
:102310001307000013173700B387E70023A0B700A7
:1023200023A2A70067800000130710006FF09FFE34
:10233000130720006FF01FFE130730006FF09FFDA2
:10234000130740006FF01FFD130750006FF09FFC54
:10235000130770006FF01FFC130760006FF09FFB06
:10236000977703009387075103A747006300E504AD
:1023700003A7C7006306E50403A747016306E50456
:1023800003A7C7016306E50403A747026306E50444
:1023900003A7C7026306E50403A74703630AE5042E
:1023A00003A7C7036302A7046780000013070000A8
:1023B00013173700B387E70023A0070067800000EA
:1023C000130710006FF0DFFE130720006FF05FFEB1
:1023D000130730006FF0DFFD130740006FF05FFD63
:1023E000130750006FF0DFFC130770006FF05FFC05
:1023F000130760006FF0DFFB130101FF232481004E
:10240000232291002320210113040500232611001B
:102410009384050013090600EF20100A03274404E3
:102420009307F0FF6314F7002322040403278404B6
:102430009307F0FF6314F70023240404EF20100B2C
:1024400083278403639A0700130609009385040019
:1024500013054402EF208024EF2010068327840414
:10246000635AF004832744026386070493044402FA
:102470006F000002832784049387F7FF2324F4046A
:10248000832784046358F00283274402638407028D
:1024900013850400EF204031E30E05FCEF20005EC1
:1024A000832784049387F7FF2324F4048327840479
:1024B000E34CF0FC9307F0FF2324F404EF20100317
:1024C000EF20807F83274404635AF00483270401AC
:1024D00063860704930404016F0000028327440409
:1024E0009387F7FF2322F404832744046358F00200
:1024F000832704016384070213850400EF20C02AA8
:10250000E30E05FCEF208057832744049387F7FFF1
:102510002322F40483274404E34CF0FC9307F0FFE8
:102520002322F404032481008320C100832441007A
:1025300003290100130101016F20407B63020504A0
:10254000130101FD232E3101232C41012326110209
:10255000138A0700232481022322910223202103CE
:10256000232A51012328610123267101930790003A
:102570009309070063FAE700737004306F000000EE
:10258000737004306F000000130B05009384050086
:1025900013090600938B0600930A08006302082CB7
:1025A00013050006EF305059130405006302052A95
:1025B0001319290023285503130609009305500A0F
:1025C00013850A00EF40C00903C7040083270403F2
:1025D0001309C9FF230AE40203C704003389270152
:1025E0001379C9FF6306070E83C71400A30AF40218
:1025F00083C71400638E070C83C72400230BF402E7
:1026000083C724006386070C83C73400A30BF4023E
:1026100083C73400638E070A83C74400230CF40287
:1026200083C744006386070A83C75400A30CF402DF
:1026300083C75400638E070883C76400230DF40228
:1026400083C764006386070883C77400A30DF40280
:1026500083C77400638E070683C78400230EF402C9
:1026600083C784006386070683C79400A30EF40221
:1026700083C79400638E070483C7A400230FF4026A
:1026800083C7A4006386070483C7B400A30FF402C2
:1026900083C7B400638E070283C7C4002300F40419
:1026A00083C7C4006386070283C7D400A300F40471
:1026B00083C7D400638E070083C7E4002301F404BA
:1026C00083C7E4006386070083C7F400A301F40412
:1026D000930A440013850A00A3010404232634034B
:1026E00023283405232A0404EFE0CFDC13058401FA
:1026F000EFE04FDC9307A000B3873741232C04049D
:1027000023288400232CF40023228402232204049F
:10271000232E040413860B0093050B0013050900F8
:10272000EFD01FFC2320A40063040A0023208A00AA
:102730007370043017E90100130909E183270900C8
:1027400097E40100938404E2638C070003A704006C
:1027500083A7040083274704938717002322F704E5
:1027600017E70100130707DF832707009387170088
:1027700097E6010023A0F6DE83A70400638E070E10
:102780008327090017EB0100130BCBF1639C0700B3
:1027900083A7040083A7C70263E6F90097E7010057
:1027A00023A287DC97E70100938707D983A7070057
:1027B00017E70100130787D90325C4020327070081
:1027C0009387170097E6010023A8F6D62324F40484
:1027D0006376A70097E7010023AAA7D693054001D7
:1027E000EF60405793850A003305AB00EFE00FCD53
:1027F000832709006388070083A7040083A7470491
:10280000639C07088327090013041000638A0700EC
:1028100083A7040083A7C70263F43701EFD05FD713
:10282000130504008320C102032481028324410292
:10283000032901028329C101032A8101832A41015D
:10284000032B0101832BC1001301010367800000EA
:1028500013850A00EF3050461304F0FF6FF05FFC61
:1028600013152600EF30502D930A0500E31A05D208
:102870001304F0FF6FF0DFFA97E7010023A487CE7F
:102880000327070093071000630AF70217EB010004
:10289000130B4BE16FF01FF103A7040083A60400A4
:1028A000832747049387F7FF2322F70483A746046F
:1028B000E39A07F4736004306FF0DFF4130A00004A
:1028C00017EB0100130B0BDE930BA00013050A009E
:1028D00093054001EF600048130A1A003305AB006E
:1028E000EFE04FBBE3147AFF97EB0100938B0BE80B
:1028F00013850B00EFE00FBA17EA0100130A4AE84C
:1029000013050A00EFE00FB917E50100130585E88C
:10291000EFE04FB817E50100130505E9EFE08FB7C9
:1029200017E50100130585E9EFE0CFB697E7010051
:1029300023A877C397E7010023A247C36FF09FE660
:10294000130101FF2324810023261100232291007B
:1029500023202101130405007370043097E4010063
:10296000938484BE83A70400639E07106318040049
:1029700097E70100938707BF03A4070013094400EA
:1029800013050900EFE0CFBB8327840263860700AD
:1029900013058401EFE0CFBA9305090017E50100A4
:1029A000130585E0EFE08FB197E701009387C7BA81
:1029B00003A7070097E70100938707B883A70700DD
:1029C0001307170097E6010023A8E6B803A7040041
:1029D0009387170097E6010023A0F6B6630C070063
:1029E00097E70100938707B803A707000327470469
:1029F000631C070E83A70400638A070697E701009C
:102A0000938747B603A707006302871073700430EB
:102A100003A704006318070817E70100130747B46A
:102A20008326070083A606006392060A1307F0FFB9
:102A300097E6010023A0E6B003A70400630807029D
:102A400003A70700032747046302070203A7070041
:102A500083A60700832747049387F7FF2322F70401
:102A600083A7460463940700736004308320C10089
:102A70000324810083244100032901001301010183
:102A80006780000097E701009387C7AD03A70700A1
:102A900083A7070083274704938717002322F7049F
:102AA0006FF0DFEC83A6070003A7070003A7460427
:102AB0001307170023A2E60417E70100130747AA2C
:102AC0008326070083A60600E38206F60327070095
:102AD0000327C7000327C7000327470097E6010025
:102AE00023AAE6A46FF05FF503A7070083A60700FB
:102AF000832747049387F7FF2322F70483A746041D
:102B0000E39A07EE736004306FF0DFEE97E70100A1
:102B1000938707A283A707006386070073700430BA
:102B20006F000000032481008320C1008324410042
:102B300003290100130101016FD09FA56304050C57
:102B400017E70100130707A2832607009307000079
:102B50006386A60A130101FF2326110023248100A6
:102B6000232291007370043097E601009386C69D7E
:102B700083A70600638C070003260700832707004E
:102B800083274604938717002322F60483A70600B1
:102B90009304050003244501638807008327070089
:102BA00083A747046394070697E701009387479B31
:102BB00083A70700638C870697E701009387079A2E
:102BC00083A707006384870697E70100938707BF01
:102BD0006306F40497E70100938707BD630CF402D2
:102BE000930710008320C100032481008324410047
:102BF000138507001301010167800000138507009A
:102C000067800000737004306F000000EF60802A5E
:102C10006FF09FF9930740006FF0DFFC83A78402F9
:102C200093B71700938727006FF0DFFB930720000F
:102C30006FF05FFB7370043097E701009387C790D4
:102C400003A70700631607026304050483A70700B0
:102C50000325C502638C070097E7010093878790DF
:102C600003A7070003274704631C070267800000CF
:102C700017E701001307078F8326070003270700C4
:102C800003A746041307170023A2E604E31005FC7C
:102C900017E701001307078D032507006FF01FFBDF
:102CA00003A7070083A60700832747049387F7FF3E
:102CB0002322F70483A74604E39A07FA73600430DB
:102CC00067800000130101FF232481001304050025
:102CD00023261100EFD01FA06318040097E701001E
:102CE0009387478803A407000324C402EFD01F9EE4
:102CF0008320C10013050400032481001301010196
:102D0000678000009307900063F6B700737004308B
:102D10006F000000130101FE232C8100232E1100FF
:102D2000232A910023282101232631012324410154
:102D3000130405007370043017E901001309C980FA
:102D40008327090063920710630004128327040598
:102D5000638EF50A17E701001307C78063F0B70217
:102D600083260700638E8612032707008324C70289
:102D7000B3B4950093C414006F00000183240700CE
:102D8000B384844093B414000327C4026386E70E1F
:102D9000832784012328B40463C807009307A00095
:102DA000B385B740232CB40093172700B387E700FF
:102DB0000327440197E901009389C98E939727005F
:102DC000B387F9006310F704130A440013050A00DF
:102DD000EFD01FF797D70100938747770325C402E9
:102DE00083A7070063F6A70097D7010023A0A77663
:102DF00093054001EF50107693050A003385A90032
:102E0000EFD0DFEB63840400EFD08FF88327090055
:102E1000638C070097D701009387C77483A70700C7
:102E200083A74704639E07048320C1010324810113
:102E300083244101032901018329C100032A810060
:102E4000130101026780000097D701009387877103
:102E500003A7070083A7070083274704938717006A
:102E60002322F704E31404EE97D701009387876FBA
:102E700003A407006FF09FED2326B4026FF05FF10B
:102E8000032481018320C10183244101032901011D
:102E90008329C100032A8100130101026F608001B0
:102EA000930400006FF05FEE630A0508130101FE52
:102EB000232A910097D401009384C46A83A7040055
:102EC000232E1100232C81002328210123263101E8
:102ED0006388A7047370043017D901001309C96609
:102EE00083270900638C070003A7040083A704005D
:102EF00083274704938717002322F70403274501FC
:102F000097E701009387878B630EF70283270900F9
:102F10006388070083A7040083A74704639E07080C
:102F20008320C1010324810183244101032901017C
:102F30008329C1001301010267800000737004300F
:102F40006F0000008327850217E7010013078784BD
:102F5000E38EE7FAE39C07FA9309450013040500A2
:102F600013850900EFD0DFDD97D701009387075E57
:102F70000325C40283A7070063F6A70097D70100C3
:102F800023A6A75C93054001EF50D05C97D70100C2
:102F9000938747713385A70093850900EFD01FD22F
:102FA00083A704000327C40283A7C702E360F7F6E0
:102FB000EFD00FDE6FF09FF5032481018320C10164
:102FC00083244101032901018329C1001301010266
:102FD0006F50506E63020506130101FE232C810021
:102FE000232A91002326310113040500232E11000A
:102FF00023282101EFD00FEE0327440197D70100CA
:103000009387C77B9309050093040000630AF702C6
:1030100013850900EFD08FEB8320C10103248101C8
:103020001385040003290101832441018329C10080
:103030001301010267800000737004306F0000000C
:103040008327840217D501001305C574E382A7FC0A
:10305000E39007FC97D701009387874D83A707006C
:103060006394070697D701009387C74F83A707008C
:103070008324C4021309440083A7C702130509006F
:10308000B3B4F400EFD0DFCB97D701009387074CA0
:103090000325C40283A7070093C4140063F6A700A6
:1030A00097D7010023A4A74A93054001EF50904A07
:1030B00097D701009387075F930509003385A70021
:1030C000EFD0DFBF6FF0DFF493058401EFD01FBFB7
:1030D0006FF01FF4130101FE37150000232E1100BD
:1030E000232C8100232A910023282101232631014A
:1030F000232441012322510123206101EF30C02309
:10310000630805229304050013050006EF30C02272
:103110001304050063040526371600009305500AC2
:103120002328950213850400EF3080538324040381
:10313000B71700009387C7FFB384F400B7474C4527
:1031400093879744130A4400232AF40213050A00C4
:10315000230C0402A30104042326040223280404EC
:10316000232A0404EFD01FB513058401EFD09FB4C8
:103170009307A000232C040493F4C4FF23288400A5
:10318000232CF4002322840223220404232E04048B
:1031900013060000971500009385C5EA1385040007
:1031A000EFD00FD42320A4007370043017D901008E
:1031B000130989398327090097D401009384843A3D
:1031C000638C070003A7040083A704008327470438
:1031D000938717002322F70417D7010013078737B7
:1031E000832707009387170097D6010023A4F6369C
:1031F00083A704006388070A8327090097D9010081
:103200009389494A639C070083A7040083A7C702E8
:103210006396070097D7010023A6873497D701004C
:103220009387873103A7070097D60100938606325C
:103230008327C40283A606001307170017D60100D0
:10324000232CE62E2324E40463F6F60017D70100AE
:10325000232EF72E139527003305F50013152500AF
:1032600093050A003385A900EFD05FA583270900E5
:103270006388070083A7040083A74704639E070CA5
:10328000832709006384070083A70400EF20500709
:1032900093071000630AF510631C0508737004306F
:1032A0006F00000097D7010023AE872A032707008D
:1032B0009307100097D901009389C93EE310F7F6F0
:1032C000938A090017DB0100130B4B4A13850A0090
:1032D000938A4A01EFD01F9CE31A5BFF17D50100C8
:1032E0001305C548EFD01F9B97DA0100938A4A491E
:1032F00013850A00EFD01F9A17D5010013058549E1
:10330000EFD05F9917D501001305054AEFD09F98BC
:1033100017D501001305854AEFD0DF9797D7010035
:1033200023A0672597D7010023AA57236FF01FEF2B
:103330008320C10103248101832441010329010168
:103340008329C100032A8100832A4100032B010045
:10335000130101026780000003A7040083A6040094
:10336000832747049387F7FF2322F70483A74604A4
:10337000E39807F0736004306FF09FF0032481013D
:103380008320C101032901018329C100032A81008F
:10339000832A4100032B010013850400832441018B
:1033A000130101026F304011737004309307F0FF76
:1033B00017D701002320F7180324810197D70100B4
:1033C00023A4A7188320C1018324410103290101FB
:1033D0008329C100032A8100832A4100032B0100B5
:1033E00097D7010023A60716130101026FC09FFFA4
:1033F0007370043097D7010023A807146FD0CF90C3
:1034000017D701001307C7128327070093871700F8
:103410002320F700678000007370043097D7010005
:103420009387871203A707006318070217D70100C5
:10343000130707120325070083A70700638C070003
:1034400097D701009387071203A7070003274704B4
:10345000631407026780000017D701001307871065
:10346000832607000327070003A746041307170056
:1034700023A2E6046FF09FFB03A7070083A60700C3
:10348000832747049387F7FF2322F70483A7460483
:10349000E39207FC7360043067800000130101FFB2
:1034A0002326110023248100EFD0CFA297D701005B
:1034B0009387070A03A40700EFD04FA18320C10020
:1034C000130504000324810013010101678000003B
:1034D00097D701009387070803A5070067800000BE
:1034E000130101FD232611022324810223229102CC
:1034F00023202103232E3101232C4101232A5101B2
:10350000232861012326710197D701009387470281
:1035100083A70700639A070617D70100130747031D
:10352000832707009387170097D6010023A2F6028E
:10353000832A0700638A0A0A97D70100938787FFC7
:1035400083A707009304000063FEFA0A97D90100DD
:103550009389491517DA0100130ACA0083270A0064
:103560009306100003A7C70293172700B387E7004D
:1035700093972700B389F90083A7090063F4F60243
:10358000930410006F00000297D70100938787FB18
:1035900083A70700930400009387170017D7010043
:1035A0002322F7FA97D70100938787F983A70700AB
:1035B00063840700930410008320C1020324810266
:1035C0001385040003290102832441028329C101D8
:1035D000032A8101832A4101032B0101832BC100AE
:1035E000130101036780000017D40100130444F79E
:1035F0008327040083A707006388070C73700430D7
:103600006F00000017D40100130484F597D901005E
:103610009389490917DA0100130ACAF417DB01007C
:10362000130BCBF28327040083A7070063800708EE
:103630008327040083A7C70003A9C7008327490085
:10364000930B490013850B0063EAFA06EFD04FEFA6
:10365000832789021305890163840700EFD04FEEA9
:103660008327C90203270B0093850B0013952700BE
:103670003305F500131525003385A9006376F7009F
:1036800017D701002324F7ECEFD04FE383270A007C
:103690000327C90283A7C702E366F7F8832704005C
:1036A0009304100083A70700E39407F89307F0FF43
:1036B00017D701002320F7E86FF05FEA17D7010062
:1036C000232AF7E66FF09FE917D70100130707E9F0
:1036D000832704000327070097D6010023A2E6E80A
:1036E00017D70100232CF7E697D70100938707E54A
:1036F00083A707009387170017D701002320F7E45B
:103700008327040083A70700639A07009307F0FF4D
:1037100017D701002320F7E26FF01FE28327040090
:1037200083A7C70083A7C70083A7470017D7010057
:103730002322F7E06FF05FE097D70100938747DF20
:1037400003A7070063160700737004306F000000C2
:10375000130101FE232E1100232C8100232A910046
:103760002328210123263101232441012322510151
:10377000232061017370043097D401009384C4DC6A
:1037800003A704006310071203A707001307F7FF3E
:1037900097D6010023AEE6D883A70700639E070AE9
:1037A00097D70100938707DB83A707006386070A83
:1037B00097DA0100938A0AEF17DA0100130A0AD98F
:1037C00017D90100130909DA930910006F00C0012D
:1037D0003385EA00EFD08FCE832709000327C40288
:1037E00083A7C7026374F70683A70A0F6380070ED7
:1037F00083A7CA0F03A4C70013058401EFD04FD4D9
:10380000130B440013050B00EFD08FD38327C402A2
:1038100083260A0093050B00139527003305F50056
:1038200013152500130705003385AA00E3F2F6FA05
:1038300017D70100232CF7D0EFD04FC883270900FA
:103840000327C40283A7C702E360F7FA97D70100F2
:1038500023A837CF6FF05FF91304000083A704009B
:10386000638C070097D701009387C7CF83A7070012
:1038700083A7470463980704130504008320C1014C
:103880000324810183244101032901018329C1000B
:10389000032A8100832A4100032B01001301010246
:1038A0006780000017D701001307C7CB83260700E6
:1038B0000327070003A746041307170023A2E60403
:1038C0006FF09FECEF50005F6FF01FFB17D401000B
:1038D000130444C783270400638C07028327040072
:1038E0001309100063860702EFF09FBF630605000F
:1038F00097D7010023A627C5832704009387F7FFE6
:1039000017D701002320F7C483270400E39E07FC98
:1039100097D701009387C7C203A70700930710003A
:10392000E31CF7F2EFC0DFC6130410006FF01FF3C3
:103930006304050263960500737004306F00000095
:1039400017D701001307C7BE83270700638A070044
:10395000737004306F000000737004306F0000005B
:10396000130101FF23248100232611008326070071
:10397000032705009386160017D60100232AD6BA1E
:1039800097D601009386C6BC83A606003304B70011
:103990002320850063F0E6046372E40263F086028C
:1039A00097D70100938707BC03A5070013054500BF
:1039B000EFD00FB913050400EF504047EFF0DFD709
:1039C000630E05008320C10003248100130101015F
:1039D00067800000E366E4FC6FF05FFC0324810075
:1039E0008320C100130101016FC09FBA630E05005F
:1039F00017D701001307C7B38327070063880700A1
:103A0000737004306F0000006FC09FB8130101FF96
:103A100023261100232481000327070093070500B4
:103A20001307170097D6010023A4E6B097D601002C
:103A3000938646B317D70100130787B10327070002
:103A400003A506003304F70013054500EFD04FAF80
:103A500013050400EF50803DEFF01FCE631A050000
:103A6000032481008320C100130101016FC05FB2F4
:103A70008320C1000324810013010101678000003D
:103A8000130101FF232481002326110097D7010091
:103A9000938707AA83A707001304000093871700E2
:103AA00017D701002326F7A897D70100938787AA85
:103AB00083A7070063EEF51417DE0100130E4ECA4C
:103AC00097D20100938242BD130400001307000047
:103AD000930F10001303500A6F00C000130ECEFEA8
:103AE0006384C20F83278EFF93060700E38807FED7
:103AF0008327CEFF83A74700232EFEFE6386C713CE
:103B000003AFC70083A747003307E500930E00000B
:103B1000232EFEFE6380C70983A8C700938748034E
:103B2000232017012322F70083A788042326F70107
:103B30002324F70083A7C8022328F70083A70805DA
:103B4000232C0700232AF70003A808038347080053
:103B500063986704930708009387170083C60700DC
:103B6000B3850741E38A66FE93D525009395050149
:103B700093D50501231EB700938E1E00130707027D
:103B8000630A1F038327CEFF83A74700232EFEFE71
:103B9000E394C7F983274E00232EFEFE6FF0DFF774
:103BA00093050000231EB700938E1E001307070223
:103BB000E31A1FFD3304D40113175400130ECEFE75
:103BC00093060700E390C2F397D7010093874799C4
:103BD00003AE070083270E006396071297D70100F4
:103BE0009387C79703AE070083270E00639A071CCD
:103BF00017DE0100130E0EAB83274E10639C0702E5
:103C000083278E11639C0726630406002320060089
:103C1000EFF09FB2130504008320C100032481004C
:103C2000130101016780000083274E00232EFEFE52
:103C30006FF01FED83278E1017DF0100130F4FB7B2
:103C400083A7470017D701002322F7B66386E73D15
:103C500083A2C70083A74700B306D500930E0000D8
:103C600017D701002324F7B4930F40001303500A21
:103C70006382E70983A8C7009387480323A016013E
:103C800023A2F60083A7880423A6F60123A4F60046
:103C900083A7C80223A8F60083A7080523AC060063
:103CA00023AAF60003A8080383470800639A673233
:103CB000930708009387170003C70700B3850741E0
:103CC000E30A67FE93D725009397070193D707016F
:103CD000239EF600938E1E0093860602638C12319B
:103CE00083278E1083A7470017D701002320F7AC46
:103CF000E392E7F983270E1117D701002328F7AACB
:103D00006FF05FF783274E00130F8E0083A64700E6
:103D10002322DE006380E633B307E50003A74600F5
:103D200083A2C600930E00002322EE00930F200012
:103D30001303500A6300EF088328C7001387480362
:103D400023A0170123A2E70003A7880423A6F701F5
:103D500023A4E70003A7C80223A8E70003A70805D8
:103D600023AC070023AAE70003A8080303470800C1
:103D7000631E672213070800130717008346070016
:103D8000B3050741E38A66FE13D725001317070121
:103D900013570701239EE700938E1E0093870702A7
:103DA0006380122383264E0003A746002322EE00E1
:103DB000E314EFF80327CE002322EE006FF0DFF7C5
:103DC00083274E00130F8E0083A747002322FE0097
:103DD000638CE72583A2C70083A74700B306D500FD
:103DE000930E00002322FE00930F20001303500ABD
:103DF0006300FF0883A8C7009387480323A0160128
:103E000023A2F60083A7880423A6F60123A4F600C4
:103E100083A7C80223A8F60083A7080523AC0600E1
:103E200023AAF60003A808038347080063986714D1
:103E3000930708009387170003C70700B38507415E
:103E4000E30A67FE93D725009397070193D70701ED
:103E5000239EF600938E1E0093860602638A121339
:103E600083274E0083A747002322FE00E314FFF8B8
:103E70008327CE002322FE006FF0DFF78327CE11C9
:103E800097DE0100938E0E9483A7470017D7010099
:103E90002328F792638AD71783AFC70083A7470009
:103EA0003307D5001303000097D6010023AAF6902C
:103EB000130F3000930220009308500A6388D7093B
:103EC00003A5C700930745032320A7002322F7007B
:103ED000832785042326E7012324F7008327C502CF
:103EE0002328F700832785026384070023265700D1
:103EF00083270505232C0700232AF7000328050341
:103F000083470800639C17059307080093871700F1
:103F100083C60700B3850741E38A16FF93D72500C0
:103F20009397070193D70701231EF700130313008C
:103F300013070702638EAF028327CE1183A74700C2
:103F400097D6010023AEF686E39CD7F783274E125F
:103F500097D6010023A6F6866FF09FF69307000020
:103F6000231EF7001303130013070702E396AFFCA9
:103F700033046400E31C06C86FF09FC99307000078
:103F8000239EF600938E1E0093860602E39A12ED9E
:103F900017CE0100130E0E7183274E103304D40187
:103FA00093165400E38E07C46FF0DFC813070000B8
:103FB000239EE700938E1E0093870702E39412DF8F
:103FC00097C701009387875903AE07003304D401D4
:103FD0009316540083270E00E38C07C06FF05FDE5A
:103FE00093070000239EF600938E1E009386060220
:103FF000E39812CF83278E113304D4019316540013
:10400000E38407C06FF09FE783274E1217C70100B4
:104010002328F77A6FF05FE883270E1117C7010096
:104020002326F7786FF0DFC28327CE002322FE001D
:104030006FF05FDA8326CE002322DE006FF0DFCD43
:10404000130101FD2322910223202103232E31019C
:10405000232C4101232A51012328610123267101C8
:10406000232611022324810297C901009389494C18
:1040700017C901001309096317CA0100130ACA4CC2
:1040800097CA0100938A0A4E97CB0100938B8B4C01
:1040900097C401009384444C130B10006F0000027E
:1040A00083A70900032449109387170017C701004D
:1040B0002320F748EFF04FE8631E040083A70400B5
:1040C000E39007FE83270900E37AFBFEEFC04FCCA5
:1040D0006FF0DFFE7370043083270A00639E0704CD
:1040E0008327091103A4C70013054400EFC05FC56F
:1040F00083A70B009387F7FF17C70100232CF74412
:1041000083A704009387F7FF17C701002326F7440E
:1041100083270A006388070083A70A0083A7470450
:104120006398070203250403EF20003913050400F8
:10413000EF2080386FF09FF803A70A0083A70A00DA
:1041400083274704938717002322F7046FF05FF952
:1041500003A70A0083A60A00832747049387F7FF73
:104160002322F70483A74604E39E07FA7360043012
:104170006FF05FFB97C701009387873B83A707001A
:10418000639E070E130101FF2326110023248100E3
:104190002322910097C7010023A4073A17C7010003
:1041A0001307473C83270700B7A6A5A59386565A51
:1041B00083A7070383A50700639ED50003A64700D6
:1041C000631AB60083A687006396C60083A7C7005C
:1041D000638AD700032507008325070093854503DD
:1041E000EF30C07617C70100130747368326070054
:1041F00017C401001304044B6F000002832707005B
:1042000063860708832707009387F7FF97C6010097
:1042100023AEF6328326070093972600B387D70094
:1042200093972700B307F40083A70700E38807FCF0
:104230000325070093172500B387A700939727004E
:104240003307F4008326470093878700B307F40001
:1042500083A4460023229700638EF40283A7C40040
:104260008320C1000324810017C70100232CF72EEF
:1042700083244100130101016780000093071000AF
:1042800017C70100232EF72A6780000073700430DF
:104290006F00000083A4440093054001EF40902B81
:1042A0003305A400232295006FF05FFB130101FE8C
:1042B00023282101232E1100232C8100232A910081
:1042C00023263101130905007370043097C40100DF
:1042D0009384842783A7040017C40100130484284F
:1042E000639C070C63140900032904009309490027
:1042F00013850900EFC0DFA48327890263860700C6
:1043000013058901EFC0DFA39385090017C50100DC
:104310001305C54AEFC09F9A83A70400638807006E
:104320008327040083A747046394070A83270400B4
:104330006384270D83A7040063820706737004302B
:1043400083A704006398070E97C70100938747214E
:1043500003A70700032707006310070C9307F0FF6C
:1043600017C701002328F71C83A7040063880702EE
:104370008327040083A747046382070203270400FE
:1043800083260400832747049387F7FF2322F7043B
:1043900083A7460463940700736004308320C1013F
:1043A0000324810183244101032901018329C100E0
:1043B0001301010267800000032704008327040023
:1043C00083274704938717002322F7046FF09FF198
:1043D0000327040083260400832747049387F7FFFD
:1043E0002322F70483A74604E39207F473600430A2
:1043F00083270400E39027F583A704006382070660
:1044000097C701009387C71283A707006388070A2D
:10441000737004306F00000083A7070083A7C700F4
:1044200083A7C70083A7470017C701002324F710FD
:104430006FF09FF3032704008327040083274704BA
:10444000938717002322F70497C70100938747112A
:1044500003A7070003270700E30207F06FF0DFFB65
:1044600097C701009387070F17C70100130787231A
:1044700083A70700032787116314F7028320C10174
:104480000324810197C7010023AE070C8324410157
:10449000032901018329C100130101026780000083
:1044A000032481018320C1018324410103290101E7
:1044B0008329C100130101026FF0DFCB03248101C6
:1044C0008320C10183244101032901018329C10003
:1044D000130101026FC0CF8B6306050A130101FFB0
:1044E0002322910097C401009384C4072320210153
:1044F0001389050083A504002326110023248100CD
:1045000093858501EFC08FFE03A5040013054500C8
:10451000EFC01F839307F0FF630AF90697C70100F6
:104520009387070303A4070003A7040083A70700DA
:104530003304240123228700636EF40697C7010029
:104540009387070203A5070083A504009385450010
:10455000EFC0CFF997C701009387C7FD83A7070076
:104560006376F40097C7010023A687FC8320C1006F
:104570000324810083244100032901001301010168
:1045800067800000737004306F00000083A5040092
:10459000032481008320C1008324410003290100FA
:1045A00017C50100130585219385450013010101FD
:1045B0006FC0CFF097C70100938747FA03A50700A4
:1045C0000324810083A504008320C10083244100CB
:1045D0000329010093854500130101016FC00FF10C
:1045E000630E050097C70100938787F483A7070030
:1045F000639A0700737004306F000000737004301A
:104600006F000000130101FF2322910097C40100F5
:10461000938444F503A704009387050083A5040051
:10462000B7060080B3E7D7002326110023248100BA
:10463000232CF7009385850113040600EFC00FE8D3
:1046400003A5040013054500EFC08FEF9307F0FFAB
:104650006304F40297C70100938787EF03A507005F
:104660008320C10083244100330585000324810099
:10467000130101016F40807B83A5040003248100A6
:104680008320C1008324410017C5010013050513D1
:1046900093854500130101016FC04FE26308050ACD
:1046A000130101FF2322910097C40100938484EB3E
:1046B000232021011389050083A50400232611006E
:1046C000232481009385850113040600EFC00FDFCA
:1046D00003A5040013054500EFC08FE69307100003
:1046E000630AF40697C70100938787E603A40700CF
:1046F00003A7040083A707003304240123228700B3
:10470000636EF40697C70100938787E503A507004A
:1047100083A5040093854500EFC04FDD97C70100D6
:10472000938747E183A707006376F40097C70100EA
:1047300023A287E08320C100032481008324410059
:104740000329010013010101678000007370043028
:104750006F00000083A50400032481008320C100B2
:10476000832441000329010017C501001305050535
:1047700093854500130101016FC04FD497C7010015
:104780009387C7DD03A507000324810083A50400E8
:104790008320C10083244100032901009385450043
:1047A000130101016FC08FD4130101FF23261100F3
:1047B00023248100232291008327C50003A4C7007E
:1047C0006304040A9304840113850400EFC04FD7E7
:1047D00097C701009387C7D583A70700639A070887
:1047E0009304440013850400EFC08FD597C70100E0
:1047F0009387C7D50327C40283A7070063F6E700A2
:1048000097C7010023A4E7D493172700B387E700D5
:104810009397270017C501001305C5E89385040089
:104820003305F500EFC08FC997C70100938787D381
:1048300083A707000327C4021305000083A7C7024C
:1048400063FAE7009307100017C70100232AF7CE89
:10485000130510008320C10003248100832441003C
:104860001301010167800000737004306F000000C5
:104870009385040017C501001305C5F1EFC00FC4EF
:104880006FF09FFA97C70100938787CA83A7070035
:1048900063960700737004306F000000130101FF7E
:1048A000232611002324810023229100B7070080D2
:1048B0000324C500B3E7F5002320F50063080408CE
:1048C000EFC00FC89304440013850400EFC04FC726
:1048D00097C70100938787C70327C40283A70700F0
:1048E00063F6E70097C7010023A2E7C693172700E6
:1048F000B387E7009397270017C50100130585DAF2
:104900003305F50093850400EFC04FBB97C7010046
:10491000938747C583A707000327C4021305000038
:1049200083A7C70263FAE7009307100017C70100C7
:104930002328F7C0130510008320C1000324810041
:10494000832441001301010167800000737004306B
:104950006F0000006304050297C70100938707BE3C
:1049600003A7070097C70100938787BE83A70700A7
:104970002320E5002322F5006780000073700430D7
:104980006F0000006304050E638E050C130101FF28
:1049900023261100232481001307050073700430BF
:1049A00097C80100938848BA83A70800638007026C
:1049B00097C70100938707BB83A6070083A707005B
:1049C00083A746049387170023A2F60417C30100A8
:1049D000130303B883A70500032603009306F0FF23
:1049E000130400006388D70417CE0100130E0EB520
:1049F00003250E0003280700832647006306A8004E
:104A0000130410006378D6023308D6401304100054
:104A10006372F80203250E00B387C7400326030024
:104A2000B387D70023A0F5002320A7002322C700C7
:104A30001304000083A70800638C070097C70100D8
:104A4000938747B283A7070083A7470463940702AD
:104A5000130504008320C100032481001301010118
:104A600067800000737004306F00000073700430C2
:104A70006F000000EF4000446FF09FFD93071000AF
:104A800017C70100232EF7AA678000006306050000
:104A90000325C5046780000013050000678000003F
:104AA000630405002326B5046780000097C7010052
:104AB000938747AB03A507006780000097C70100F5
:104AC000938787A883A7070013051000638C07004E
:104AD00097C701009387C7A503A5070013351500E5
:104AE0001315150067800000630C0508130101FE13
:104AF000232A910097C401009384C4A683A70400CD
:104B0000232E1100232C810023282101232631018B
:104B10000327C50283A7C7026376F70483278501AD
:104B200063CC070083A7040083A6C7029307A000F5
:104B3000B387D740232CF50093172700B387E700EE
:104B40000327450117C901001309C9B59397270029
:104B5000B307F9006308F70283A7040083A7C7021D
:104B60002326F5028320C10103248101832441010E
:104B7000032901018329C10013010102678000009C
:104B800067800000930945001304050013850900A0
:104B9000EFC00F9B83A7040017C701001307079BF3
:104BA0000327070083A7C7022326F4026376F700D2
:104BB00017C70100232CF798139527003305F5003C
:104BC00003248101131525008320C10183244101A1
:104BD000938509003305A9008329C1000329010138
:104BE000130101026FC08F8D63060502130101FFDF
:104BF00023261100232481002322910097C701005E
:104C00009387479603A40700630AA40073700430D7
:104C10006F00000013050000678000008327440533
:104C200063960700737004306F0000008326C4028F
:104C3000032704059387F7FF232AF4046384E6001F
:104C4000638E0700130500008320C1000324810048
:104C50008324410013010101678000009304440094
:104C600013850400EFC0CF8D0325040597C701000D
:104C70009387C78D03A707009307A000B387A740BA
:104C80002326A402232CF4006376A70097C7010013
:104C900023AEA78A93054001EF40C00B97C70100E0
:104CA000938747A03385A70093850400EFC00F8149
:104CB000130510006FF05FF97370043097C701009F
:104CC0009387878883A707006380070297C701003F
:104CD0009387478903A7070083A707008327470413
:104CE000938717002322F7046780000097C701000D
:104CF0009387878583A70700638C070297C7010006
:104D00009387478603A70700032747046302070228
:104D100003A7070083A60700832747049387F7FFAD
:104D20002322F70483A746046394070073600430CA
:104D30006780000097C701009387C78203A607001A
:104D400083A6070003A707009307A00083A6C60257
:104D500003258601B387D740232CF7006780000026
:104D600097C701009387078003A70700630A07001E
:104D700083A6070003A746051307170023AAE60426
:104D800003A5070067800000130101FD2320210314
:104D9000232611022324810223229102232E310192
:104DA000130905007370043097B401009384C4792B
:104DB00083A7040017B401001304C47A639E070A92
:104DC0008327040083A78705639A070083270400CD
:104DD0001307100023AEE704639A050E83A70400AF
:104DE000638807008327040083A74704639A071496
:104DF0007370043083A704006394070683270400BC
:104E000003A58705630805006302090483270400DE
:104E100023AC07048327040023AE070483A7040000
:104E2000638807008327040083A74704639207066B
:104E30008320C10203248102832441020329010249
:104E40008329C101130101036780000003270400C7
:104E5000832787059387F7FF232CF7046FF09FFBC9
:104E60000327040083270400832747049387170040
:104E70002322F7046FF09FF8032704008327040020
:104E800083274704938717002322F7046FF05FF30B
:104E90000327040083260400832747049387F7FF32
:104EA0002322F70483A74604E39407F873600430D1
:104EB0008320C102032481028324410203290102C9
:104EC0008329C10113010103678000000325040049
:104ED0002326B10013054500EFB09FE68325C100EE
:104EE0009307F0FF6380F50897B701009387476643
:104EF00083A907000327040083A70700B389B9002B
:104F00002322370163ECF90697B7010093874765C1
:104F100003A507008325040093854500EFB01FDD3E
:104F200097B701009387076183A7070063F6F9002D
:104F300097B7010023A03761EFB08FE56FF01FEA4C
:104F40000327040083260400832747049387F7FF81
:104F50002322F70483A74604E39C07E87360043028
:104F60006FF01FE98325040017C5010013050585AF
:104F700093854500EFB09FD46FF01FFC97B70100F9
:104F80009387C75D03A5070083250400938545002B
:104F9000EFB0DFD56FF05FFA130101FD232021038D
:104FA000232E310123261102232481022322910280
:104FB000232C410113890500930906007370043006
:104FC00097B401009384445883A7040017B40100E8
:104FD00013044459639C071403270400930720001B
:104FE0000327C7056304F702832704001345F5FF71
:104FF00003A787053375E50023ACA70483270400C6
:105000001307100023AEE704639A060A83A704007F
:10501000638807008327040083A747046394071667
:105020007370043083A70400639E07066388090039
:105030008327040083A7870523A0F9000327040022
:1050400093071000130500000327C705630EF70040
:10505000832704001349F9FF1305100003A78705F0
:105060003379E90023AC27058327040023AE070426
:1050700083A70400638807008327040083A74704ED
:105080006392070C8320C10203248102832441021E
:10509000032901028329C101032A810113010103AC
:1050A0006780000003270400832704008327470448
:1050B000938717002322F7046FF05FF7032504009E
:1050C0002326D10013054500EFB09FC78326C100FA
:1050D0009307F0FF638AF60C97B701009387474761
:1050E00003AA07000327040083A70700330ADA0096
:1050F000232247016368FA0C97B70100938747465C
:1051000003A507008325040093854500EFB01FBE6B
:1051100097B701009387074283A707006370FA0AD5
:1051200097B7010023A847416F00400903270400F7
:105130008327040083274704938717002322F7045B
:105140006FF09FE9032704008326040083274704A8
:105150009387F7FF2322F70483A74604E39407F21B
:10516000736004308320C10203248102832441023E
:10517000032901028329C101032A810113010103CB
:105180006780000003270400832604008327470468
:105190009387F7FF2322F70483A74604E39207E8E7
:1051A000736004306FF0DFE78325040017B501005A
:1051B0001305C56093854500EFB05FB0EFB04FBDFC
:1051C0006FF0DFE497B701009387473903A5070025
:1051D0008325040093854500EFB05FB16FF01FFE9B
:1051E000630A050C130101FF23261100232481000B
:1051F00023229100232021017370043097B4010011
:105200009384843483A704006396070863860600AA
:105210008327850523A0F600930706009306200048
:105220000326C505232ED5041387050013040500A6
:105230006382D70A63F4F608930530006388B700E9
:10524000930540006396B700630CD610232CE4044A
:1052500093071000630CF6081304100083A70400E2
:10526000638C070097B701009387C72F83A70700B8
:1052700083A7470463980706130504008320C10031
:10528000032481008324410003290100130101014B
:105290006780000097B701009387C72C03A707001A
:1052A00083A7070083274704938717002322F70467
:1052B0006FF0DFF5737004306F000000930610008C
:1052C000E398D7F88327850533E7B700232CE50457
:1052D0006FF01FF88327850593871700232CF504AB
:1052E0006FF01FF7EF30103D6FF01FF91309440006
:1052F00013050900EFB0DFA497B7010093870725D6
:105300000325C40283A7070063F6A70097B701002F
:1053100023AEA72293054001EF30D02397B70100B9
:10532000938747383385A70093050900EFB01F998D
:105330008327840263860700737004306F000000C7
:1053400097B701009387072283A707000327C402AA
:1053500083A7C702E3F2E7F0EFB08FA36FF0DFEFB0
:10536000130400006FF09FEF63080508130101FEAE
:10537000232C8100232A9100232821012326310197
:105380002324410123225101232E110093090700F8
:10539000138A060093040600138905001304050010
:1053A000EFB04FB3930A050063060A008327840514
:1053B0002320FA000327C40593072000232EF404BA
:1053C0006380F40463FA9710930630006388D40076
:1053D000930640006396D400630CF70E232C24053B
:1053E000930710006312F70A83278402638207027F
:1053F000737004306F000000737004306F000000A1
:105400008327840593871700232CF4046FF05FFD36
:1054100097B701009387C71183A707006390070A16
:105420009304440013850400EFB09F9197B70100E7
:105430009387C7110325C40283A7070063F6A7005B
:1054400097B7010023A4A71093054001EF309010F7
:1054500097B7010093870725938504003385A7003C
:10546000EFB0DF8597B701009387C70F83A70700C9
:105470000327C40283A7C70263F8E7006386090015
:105480009307100023A0F9001304100013850A00ED
:10549000EFB0CFA3130504008320C10103248101D1
:1054A00083244101032901018329C100032A8100CA
:1054B000832A4100130101026780000093058401E3
:1054C00017B501001305052DEFB04FFF6FF09FF9E1
:1054D000130400006FF09FFB93071000E392F4F0B9
:1054E0008327840533E92701232C24056FF05FEF20
:1054F000630A050E130101FE232C8100232A91006B
:105500001304050023263101232E11002328210135
:1055100093840500EFB00F9C930720008326C405F9
:10552000232EF40483278405130710009309050034
:1055300093871700232CF4046396E60883278402DC
:1055400063860700737004306F00000097B7010096
:10555000938707FE83A70700639A0708130944008F
:1055600013050900EFB0CFFD97B70100938707FE41
:105570000325C40283A7070063F6A70097B70100BD
:1055800023A6A7FC93054001EF30C07C97B701002C
:1055900093874711930509003385A700EFB00FF2F9
:1055A00097B70100938707FC83A707000327C4026E
:1055B00083A7C70263F8E70063860400930710001F
:1055C00023A0F400032481018320C101832441012D
:1055D00003290101138509008329C1001301010278
:1055E0006FB0CF8E737004306F000000930584019C
:1055F00017B501001305051AEFB04FEC6FF05FFA15
:1056000093070500630805067370043017B701009F
:10561000130787F383260700639E060203A6C705C8
:1056200093062000130500006316D60023AE07047E
:105630001305100083270700638C070097B701004C
:10564000938747F203A7070003274704631C070259
:105650006780000097B601009386C6F003A6060097
:1056600083A6060083264604938616002322D604CA
:105670006FF0DFFA97B701009387C7EE83A70700A3
:105680006FF09FF803A7070083A60700832747044E
:105690009387F7FF2322F70483A74604E39A07FAC8
:1056A0007360043067800000130101FB2322910422
:1056B00023202105232C4103232A5103232861039E
:1056C000232671032326110423248104232E31036E
:1056D00023248103232291032320A10317B901006E
:1056E000130949E917BB0100130B0BE897B401003C
:1056F0009384C4E797BA0100938A8AE7130A1000DB
:10570000930B90008327090003A707006306071681
:1057100083A7C70083A90700EFD09FCEEFD0DFCFCC
:1057200083270B00130C05006368F50C97B7010085
:1057300023ACA7E2130600006376352303A504001B
:10574000B3858941EFC05FCBEFD01FFF630605161D
:1057500003A50400930600001306000093058100D2
:10576000EFC0CF94E30005FA83278100E3C207FE70
:105770008329010183A74901638607001385490036
:10578000EFB00FDCEFD05FC983270B00130C0500CF
:105790006362F50C8327810017B70100232687DD9C
:1057A000E3E8FBFAB317FA0013F7072163100720A9
:1057B00013F7770C6316072A93F70702E38A07F8B3
:1057C00013850900EF00504F6FF09FF883A7C700C3
:1057D00003A4C70083AC07009309440013850900A4
:1057E000EFB00FD68327440213050400E7800700BB
:1057F0008327C4016386470D8327090003A7070099
:10580000E31607FC03A70A0097B6010023AE86D56E
:1058100097B6010023AEF6D497B7010023ACE7D4C6
:10582000EFD09FF16FF0DFF283A7C70003A4C7009A
:1058300003AD0700930C440013850C00EFB04FD06C
:105840008327440213050400E78007008327C4016F
:10585000638C470B8327090003A70700E31607FCA7
:1058600003A70A0097B6010023A4F6D097B701005A
:1058700023A2E7D06FF01FF2EFD09FB8EFD0DFB9CF
:1058800083270B00130C0500E368F5F683A70A00D5
:1058900003A504009309000003A60700B38589410E
:1058A00017B70100232287CD13361600EFC0DFB4EF
:1058B000EFD09FE8E31E05E8EFA09FCD6FF05FE912
:1058C0008327840193850900B387FC0063E2FC0809
:1058D00083A7040063860702232A0100232C910179
:1058E000232E8100EFF08F9D03A504009306000096
:1058F0001306000093054101EFB0CFFBE31E05EE58
:10590000737004306F0000008327840193850C00BE
:10591000B307FD006362FD0883A7040063860702E6
:10592000232A0100232CA101232E8100EFF00F99DF
:1059300003A504009306000013060000930541012F
:10594000EFB04FF7E31805F0737004306F000000FC
:10595000032509002322F40023288400EFB00FB9A7
:105960006FF09FE9EFD05FDD8327090083A7C700B1
:1059700003A4C700930C440013850C00EFB04FBC88
:105980008327C401638A4705832744021305040063
:10599000E78007006FF0DFDB032509002322F40016
:1059A00023288400EFB08FB46FF0DFEA8327C100B3
:1059B00023ACF9006382070AB387870123A2F900A9
:1059C00023A83901938549006362FC0803A50A00F6
:1059D000EFB0CFB16FF0DFD7832784012328840095
:1059E0003387F9002322E400636AEC04330C3C4162
:1059F000636EFC0283A7040063860702232A01006A
:105A0000232C3101232E8100EFF04F8B03A50400DE
:105A1000930600001306000093054101EFB08FE9E3
:105A2000E31405F6737004306F00000003A50A004C
:105A300093850C00EFB08FAB6FF01FF503250900C5
:105A400093850C00EFB08FAA6FF01FF403250900B7
:105A5000EFB0CFA96FF0DFCF737004306F0000009C
:105A60008327C10083A6890123A839013387D70082
:105A700023A2E9006362EC06B307FC4063EAD706A1
:105A800083A7490213850900E780070083A7C9019E
:105A9000E39047CD83A689018327C10003A70400B3
:105AA000B387D70063060702232A0100232CF100E5
:105AB000232E3101EFF08F8003A504009306000030
:105AC0001306000093054101EFB0CFDEE31205C8D5
:105AD000737004306F0000006374FC00E372F7FA27
:105AE0000325090093854900EFB04FA06FF05FC612
:105AF00003A50A0093854900EFB04F9F6FF05FC583
:105B0000130101FF23248100232611002322910089
:105B10002320210117B40100130444A5EFF0CF990D
:105B20008327040063840704EFF04F9C832704005D
:105B3000638A07029308000013080000930700001F
:105B400013072000930600001306004097B50100DC
:105B50009385C58617050000130545B5EFC01F9E48
:105B600063140506737004306F00000017B901005C
:105B7000130909C613050900EFB0CF9197B40100CE
:105B8000938444C613850400EFB0CF901306000041
:105B90009305C0001305400097B7010023AC279D73
:105BA00097B7010023A6979CEFB08FBC17B70100F1
:105BB000232EA79A6306050297A501009385857F8A
:105BC000EFC04FF06FF05FF68320C1000324810027
:105BD00083244100032901001301010167800000B3
:105BE000737004306F000000638A050A130101FD21
:105BF000232A5101930A05001305C00223248102C0
:105C00002322910223202103232E3101232C410141
:105C1000232611022328610123267101130907009D
:105C200093890600130A060093840500EF00C070F4
:105C300013040500630C0502EFF00F8897B701000D
:105C40009387C79283A70700638E0704EFF00F8A3C
:105C50001305440023205401232C9400232E4401D7
:105C60002320340323222403EFB0CF841305040040
:105C70008320C102032481028324410203290102FB
:105C80008329C101032A8101832A4101032B0101D8
:105C9000832BC1001301010367800000737004307F
:105CA0006F00000097BB0100938B8BB213850B0034
:105CB000EFA05FFE17BB0100130BCBB213050B0067
:105CC000EFA05FFD130600009305C0001305400020
:105CD00097B7010023A0778B97B7010023AA6789A4
:105CE000EFB00FA917B701002322A788630A0500A8
:105CF00097A501009385056CEFC0CFDC6FF01FF511
:105D0000737004306F000000630E0506130101FE7E
:105D1000232C8100232E1100232A910017B40100A7
:105D20001304C4848328040013080500130500002D
:105D300063800804930407002322B1001387060040
:105D40002324C100232601019306500063C0B6043A
:105D5000EFE0DFD693072000630EF504032504006F
:105D6000930600001306000093054100EFB08FB4C6
:105D70008320C10103248101832441011301010215
:105D800067800000737004306F00000093054100CD
:105D9000930600001306070013850800EFB05F8329
:105DA0008320C101032481018324410113010102E5
:105DB000678000000325040093060000138604009A
:105DC00093054100EFB00FAF6FF09FFA6306050037
:105DD0000325050067800000737004306F00000029
:105DE00063160500737004306F000000130101FF9B
:105DF000232611002324810013040500EFE0DFEBCC
:105E0000032544013334A000EFE05FEE13050400E6
:105E10008320C10003248100130101016780000079
:105E200063160500737004306F000000130101FF5A
:105E3000232481001304050023261100EFE0DFE78F
:105E400003240402EFE09FEA8320C100130504004D
:105E5000032481001301010167800000631605001F
:105E6000737004306F000000130101FF23248100D0
:105E700023229100138405009304050023261100BA
:105E8000EFE09FE323A08402032481008320C1006C
:105E900083244100130101016FE05FE5130101FF5D
:105EA0001305C0012324810023261100EF00C04800
:105EB00013040500630805002320050013054500B1
:105EC000EFA05FDD130504008320C10003248100DF
:105ED000130101016780000063020502B70700FF9C
:105EE000B3F7F50063860700737004306F0000009D
:105EF000639A0500737004306F0000007370043003
:105F00006F000000130101FE232C810023282101D2
:105F1000232631012324410123225101232E110084
:105F2000232A91009309070013890600930A0600AB
:105F300013840500130A0500EFE05FB8631805003D
:105F400063860900737004306F000000EFD04FCB00
:105F500083240A00B3779400631209046382070460
:105F600063880A009347F4FFB3F797002320FA00F1
:105F7000EFD08FFC8320C10103248101138504002D
:105F800003290101832441018329C100032A8100DF
:105F9000832A41001301010267800000E302F4FC40
:105FA000E38809FCB3355001939585016306090028
:105FB000B7070004B3E5F50013860900B3E58500D3
:105FC00013054A00EFE0CFE1EFD00FF763140500AF
:105FD000EFA00FDCEFE01FD69317650093090500D3
:105FE00063DA0700B70400019384F4FFB3F4990067
:105FF0006FF05FF8EFE05FCC83290A00B3773401DC
:1060000063100902638A070063880A009347F4FF5C
:10601000B3F737012320FA00EFE05FCD6FF09FFC6C
:10602000E31CF4FE6FF05FFE630C0500B70700FF92
:10603000B3F7F500638A0700737004306F00000047
:10604000737004306F000000130101FF23248100EE
:10605000130405002326110023229100232021018F
:1060600013890500EFE05FC5832404009345F9FF21
:10607000B3F795002320F400EFE05FC78320C10051
:1060800003248100138504000329010083244100B7
:106090001301010167800000130101FF2324810027
:1060A0001304050023261100EFA0CFE2032404000F
:1060B000EFA0CFE18320C100130504000324810079
:1060C0001301010167800000630C0500370700FF22
:1060D000B3F7E500638A0700737004306F000000B7
:1060E000737004306F0000006F20905FB70700FFEF
:1060F000B377F60063860700737004306F0000000A
:1061000063160600737004306F000000130101FE77
:10611000232C81002328210123263101232441013E
:10612000232E1100232A910013890600938905006C
:10613000130A050013040600EFE05F98631E0504D0
:1061400063060900737004306F000000EFD04FAB9E
:1061500083240A009385090013050A00B3E499001B
:10616000EFF09FF6B3779400630AF40883240A00E3
:10617000EFD08FDC8320C10103248101138504004B
:1061800003290101832441018329C100032A8100DD
:106190001301010267800000EFD08FA683240A005C
:1061A0009385090013050A00B3E43401EFF0DFF131
:1061B000B3F7840063848704E30A09FAB70500058E
:1061C00013060900B365B40013054A00EFE04FC1A0
:1061D000EFD08FD663140500EFA08FBBEFE09FB523
:1061E000931765009304050063D40702B707000105
:1061F0009387F7FFB3F4F4006FF0DFF783270A000B
:106200001344F4FFB3F787002320FA006FF05FF622
:10621000EFE09FAA83240A00B37794006398870075
:106220009347F4FFB3F797002320FA00EFE01FAC89
:106230006FF0DFFB130101FF2324810023261100EF
:106240001304050023229100EFD08F9B8327440085
:1062500063860702032504019304C40063189500B4
:106260006F0080030325040163089502B70500024F
:10627000EFE04FE183274400E39607FE1305040097
:10628000EF008023032481008320C1008324410088
:10629000130101016FD04FCA737004306F0000000A
:1062A000630C0500370700FFB3F7E500638A0700BA
:1062B000737004306F000000737004306F000000D2
:1062C0006F201042630C0500B70700FFB3F7F5001D
:1062D000638A0700737004306F000000737004302D
:1062E0006F000000130101FF23248100232291008D
:1062F000232611001304050093840500EFE0DF9BC3
:106300000327040093C7F4FFB377F7002320F400BA
:10631000032481008320C100832441001301010173
:106320006FE0DF9C630605000325850167800000A0
:106330001305000067800000130101FF2324810082
:106340002326110013040500EFD08F8B97A70100BF
:106350009387872283A70700639C0704B7970100F0
:1063600017A70100130787499387C7FF97A6010066
:1063700023AAE62017A701002324F72017A701006E
:106380002320F74897A701009387471F17A701000D
:106390002326F7469307100017A701002326071EA0
:1063A00017A70100232C071C17A701002326F71CA1
:1063B00063120402EFD04FB8EF10805813040000AE
:1063C000130504008320C10003248100130101018F
:1063D0006780000013058400937735006398070CED
:1063E000B79701001307F5FF9387A7FFE3E4E7FCE6
:1063F00097A601009386061983A706006F00400147
:1064000003A70700630A07009386070093070700A6
:1064100003A74700E366A7FE17A7010013070716A7
:10642000E38AE7F803A70700130600011384870037
:1064300023A0E60003A74700B306A740637ED60269
:106440003388A7002322D80023A2A7008325480071
:1064500097A60100938606136F008000930607003D
:1064600003A7060003264700E36AB6FE2320E800E0
:1064700023A0060103A7470097A70100938787126F
:1064800083A70700B387E74017A70100232CF71065
:10649000EFD08FAAE30204F2130504008320C100A9
:1064A0000324810013010101678000001375C5FFFB
:1064B000130545006FF0DFF263080506130101FFC5
:1064C000232481002326110013040500EFC05FF38D
:1064D000930584FF0326C4FF17A701001307870A4B
:1064E0006F008000138707008327070083A64700FB
:1064F000E3EAC6FE232CF4FE2320B70097A7010091
:106500009387470A03A707008327C4FF032481005A
:106510008320C100B387E70017A701002324F708F1
:10652000130101016FD04FA16780000097A7010000
:106530009387470703A50700678000006780000076
:106540003367B5001377370093070500631207041C
:106550009308D6FFB30815011307050093860500BD
:106560006378150303A806001307470093864600C7
:10657000232E07FFE36817FF9347F5FFB387170143
:1065800093F7C7FF93874700B385F500B307F5007E
:106590003306C50063F4C70C938645001388470093
:1065A000B3B6D70033B8050133E7F50093C616003C
:1065B0001348180013773700B3E6060113371700A6
:1065C0003377D700330EF64093861700630807062B
:1065D0001337AE006314070613532E00138805000B
:1065E000938607001307000083280800130717008D
:1065F0001308480023A0160193864600E36667FE51
:106600001377CEFFB385E500B387E7006306EE049A
:1066100083C60500138717002380D700637EC70257
:1066200083C6150013872700A380D7006376C702AF
:1066300003C725002381E70067800000B307F64009
:10664000B387F5009385150003C7F5FF9386160001
:10665000238FE6FEE398F5FE678000006780000068
:10666000B367C50093F73700B308C5006382070E10
:1066700063761511B307A04093F7370013873700EF
:106680009306500093F5F50F130815003383A840C7
:106690001306F6FF6374D700130750006368E60E15
:1066A0006380070E2300B50013071000638EE70018
:1066B000A300B50013073000130825006396E70018
:1066C000130835002301B5001396850033E6C50095
:1066D000139705013367E6003303F3409396850172
:1066E000B366D70013562300B307F5001307000065
:1066F00023A0D7001307170093874700E36AC7FE5C
:106700001377C3FFB307E8006300E3082380B700F3
:1067100013871700637C1703A380B7001387270034
:10672000637617032381B70013873700637017035D
:10673000A381B70013874700637A17012382B7004C
:106740001387570063741701A382B70067800000A6
:1067500093F5F50F13978500B365B70013970501FF
:106760003367B700E37415FF93070500938747006D
:1067700023AEE7FEE3EC17FF6780000067800000B0
:10678000130805006FF05FF46780000093070500B1
:106790006FF0DFF78347050013070500638C0700E0
:1067A0001305150083470500E39C07FE3305E5400C
:1067B00067800000130500006780000013051500C6
:1067C0008347F5FF9385150003C7F5FF638807002E
:1067D000E386E7FE3385E74067800000930700000B
:1067E0006FF05FFF930705009385150003C7F5FF62
:1067F00093871700A38FE7FEE31807FE678000006A
:1068000083460500930700026398F6001305150000
:1068100083460500E38CF6FE938756FD93F7D70F6A
:10682000638007049307050093050000638806044E
:106830001305000093871700138606FD1317250024
:1068400083C607003305A700131515003305A600FE
:10685000E39206FE638405003305A04067800000D4
:10686000938536FD8346150093B5150093071500F3
:10687000E39006FC130500006FF0DFFD1305000038
:106880006780000083A705002380A70083A7050079
:106890009387170023A0F5006780000097A60100EA
:1068A0009386C6CE83A7060017370300130787F524
:1068B00013861700B307F7002380A70097A50100F0
:1068C00023A6C5CC9307A000630AF5009307000434
:1068D0006308F6001305000067800000E30C06FE65
:1068E000370610F0130717008347F7FF2320F6F051
:1068F00083A706009387F7FF97A5010023A8F5C893
:10690000E39207FE1305000067800000130101EB0E
:106910002322911423202115232A51132324811388
:106920002326111423248114232E3113232C4113E5
:106930002328611323267113232291132320A113EB
:10694000232EB11193040500138905002326C100ED
:10695000130C5002930A9000834709006388870351
:10696000638C070603A404006F008000638607069B
:106970002300F40003A404001309190013041400F5
:1069800023A0840083470900E39287FF0346190090
:106990009308190093860800130D00029309F0FF75
:1069A000130AF0FF13080000130550059307D6FDE6
:1069B00093F7F70F13891600636EF53A17970100E6
:1069C0001307476493972700B387E70083A707005F
:1069D000B387E700678007008320C1140324811474
:1069E00083244114032901148329C113032A811329
:1069F000832A4113032B0113832BC112032C811211
:106A0000832C4112032D0112832DC1111301011595
:106A100067800000930C800023240100930710007E
:106A200063DA071D8327C10003A40400938B77005A
:106A300093F68BFF03AB060083A94600938786007D
:106A40002326F10013860C009306000013050B00AB
:106A500093850900EF1010602328A1009307000020
:106A600063803733930D4101930B100013860C00A4
:106A70009306000013050B0093850900EF10C07FFB
:106A80009306000013860C00130B05009389050084
:106A9000EF10505C8327810023A0AD0093861B007C
:106AA000938D4D0063863701938B06006FF01FFCBA
:106AB000E37C9BFF63D24603930704002380A70176
:106AC00003A40400130AFAFF9307140023A0F400A0
:106AD00013840700E3C446FF93962B00930701013C
:106AE000B386D7006F008002938777052300F400F8
:106AF00003A40400938BFBFF93871B001304140073
:106B000023A084009386C6FFE358F0E483A7060021
:106B1000E3ECFAFC938707036FF05FFD83A70400A3
:106B2000930600030327C1002380D70083A7040036
:106B300093064700930C00011386170023A0C4009E
:106B400013068007A380C70003A4040023240100C8
:106B5000930707001304140023A0840003AB07006D
:106B6000930900002326D1006FF0DFED8327C100D9
:106B700083AC0700938B470063880C28635C402537
:106B80009307D002631EFD2083C70C0063880702B1
:106B900063D8092483A60400938C1C00130AFAFF0F
:106BA0002380F60003A404001304140023A084002F
:106BB00083C70C00E39E07FC6352400303A4040058
:106BC000930700022300F40003A40400130AFAFF51
:106BD0001304140023A08400E3160AFE2326710187
:106BE0006FF09FD72324010093071000930CA0009F
:106BF000E3CA07E38327C10003A404009386470088
:106C00006FF0DFF503C61600930609006FF01FDA78
:106C100083A70400930650022380D70003A4040036
:106C20001304140023A084006FF01FD3930C000101
:106C3000232401006FF09FDE8327C10003C61600E6
:106C40009306090083A90700938747002326F100D4
:106C5000E35E0AD4138A09009309F0FF6FF01FD591
:106C600003C61600130DD002930609006FF01FD45F
:106C70009347FAFF93D7F74103C61600337AFA0019
:106C8000930609006FF09FD203C61600130D000390
:106C9000930609006FF09FD183C51600930906FD86
:106CA00093060900938705FD13860500E3E2FAFACF
:106CB00093972900B3893701938616009399190099
:106CC000B389B90083C50600938909FD938705FD43
:106CD00013860500E3FEFAFC6FF09FF70327C1005F
:106CE00083A7040083260700130747002326E1003B
:106CF0002380D70003A404001304140023A08400FD
:106D00006FF09FC59307100063D4070F8327C1005E
:106D10009386770093F686FF938786002326F100FB
:106D200083A9460083A7060063DE090E83A604003C
:106D30001306D002B307F0402380C60003A404006A
:106D4000B336F000B30930411304140023A08400CB
:106D5000138B0700B389D940930CA00023240100B2
:106D60006FF05FCE03C616001308180093060900E3
:106D70006FF0DFC383A70400138908006FF09FE959
:106D8000E3729BCF93071000930B00009306100053
:106D9000E3C447D36FF05FD4979C0100938C8C625F
:106DA0009385090013850C00EF005075330AAA4043
:106DB0006352400303A404002300A40103A40400BD
:106DC000130AFAFF1304140023A08400E3160AFE3A
:106DD000130A000083C70C00E38207E0E3CC09DA62
:106DE0009389F9FF1307F0FFE396E9DA6FF0DFDC30
:106DF0008327C1009386470083A707002326D1007D
:106E000093D9F7416FF05FF2635640019307D002C8
:106E1000E314FDF8979C0100938CCC5A93078002F1
:106E20006FF01FD7138B0700930CA00023240100E1
:106E300003A404006FF01FC1130101EB232E3113D3
:106E4000B70900409387F9FF23248114232291146A
:106E5000232C4113232A51132326111423202115F7
:106E600023286113232671132324811323229113D2
:106E70002320A113232EB111130A05002324B100EE
:106E80001794010013048470973A0300938A8A9739
:106E9000979401009384842C2326F10093055002DB
:106EA0001305A00013080004B70610F083470A007A
:106EB000638EB7046388070A03270400130A1A00C5
:106EC000130617003387EA009798010023A0C86CC7
:106ED0002300F7006380A708E31A06FD17370300B5
:106EE00013074792130717008347F7FF23A0F6F015
:106EF000832704009387F7FF179601002328F6687D
:106F0000E39207FE83470A00E396B7FA83461A0026
:106F100013051A0013070500930B0002130BF0FF73
:106F2000130CF0FF13080000930550059308900020
:106F30009387D6FD93F7F70F130A170063ECF54418
:106F400093972700B387970083A70700B38797001D
:106F500067800700173703001307C78AE31406F892
:106F60006FF0DFF48320C1140324811483244114BF
:106F7000032901148329C113032A8113832A41138E
:106F8000032B0113832BC112032C8112832C41127A
:106F9000032D0112832DC11113010115678000001B
:106FA000930C8000130D00009307100063DA072193
:106FB000832781009387770093F787FF83AD0700CE
:106FC00003AB4700138787002324E10013860C00DE
:106FD0009306000013850D0093050B00EF1090073A
:106FE0002328A10063086D4513094101930910008E
:106FF00013860C009306000013850D0093050B000B
:10700000EF10802713860C0093060000930D0500F7
:10701000138B0500EF1010042320A9009389190099
:1070200013094900E3166DFDE3F49DFD130600040A
:10703000B70610F063D48903832704001387170071
:10704000B387FA009795010023A2E55423807701C6
:10705000630AC706130CFCFFE3C089FF8327C10046
:107060001305C10093089000B386F900939626009B
:1070700093070101B386D7001308A000130300048F
:10708000370610F0E38CA6E083A706009305000303
:1070900063F4F8009305700503270400B387B70075
:1070A000930517003387EA00179E01002320BE4E88
:1070B0002300F70063860737638C65329386C6FF2B
:1070C0006FF05FFC172703001307C7731307170040
:1070D0008347F7FF23A0F6F0832704009387F7FF89
:1070E0009795010023A4F54AE39207FE130CFCFFD9
:1070F0006FF09FF683270400130600041387170020
:107100009795010023A4E548B386FA009305000390
:107110002380B6006308C750938727009796010025
:1071200023A6F6463387EA00930680072300D7009C
:10713000172703001307076DB70610F06392C70205
:10714000130717008347F7FF23A0F6F083270400F7
:107150009387F7FF17960100232AF642E39207FE72
:1071600083278100930C0001130D000093874700D3
:1071700003278100130B0000832D07002324F10057
:107180006FF0DFE48327810083AC07001389470099
:10719000638E0C4C6358802B9307D0026394FB3EA4
:1071A00003C70C00930507006314072A6F00002F24
:1071B00093071000930CA000130D0000E3CA07DF33
:1071C00083278100938747006FF09FFA8327810010
:1071D0008346170013070A0003AB07009387470095
:1071E0002324F100E3560CD4130C0B00130BF0FF17
:1071F0006FF01FD483461700930BD00213070A00C9
:107200006FF01FD39347FCFF93D7F74183461700D6
:10721000337CFC0013070A006FF09FD183461700F0
:10722000930B000313070A006FF09FD0034617006B
:10723000138B06FD13070A00930706FD930606004D
:10724000E3E2F8FA93172B00B387670113071700DF
:1072500093971700B387C70003460700138B07FDFA
:10726000930706FD93060600E3FEF8FC6FF09FF718
:1072700083258100832704001306A00003A70500CF
:1072800093861700B387FA00179501002320D530A5
:107290002380E700138945006300C7369307000485
:1072A0006384F62A232421016FF05FBF9307100047
:1072B00063DE07358327810013877700137787FF05
:1072C000930787002324F100032B4700832707003F
:1072D00063560B3E032704001306000493061700B1
:1072E0009795010023A4D52A3387EA009305D0029D
:1072F0002300B700638CC638B307F0403337F00083
:10730000330B6041938D0700330BEB40930CA000CF
:10731000130D00006FF09FCB834617001308180071
:1073200013070A006FF0DFC08346170013070A0037
:107330006FF01FC083270400930600041387170013
:10734000179601002324E624B387FA00130650029F
:107350002380C700E314D7B4172703001307874A15
:10736000B70610F0130717008347F7FF23A0F6F0C6
:10737000832704009387F7FF179601002328F62040
:10738000E39207FE6FF09FB1930C0001130D000014
:107390006FF09FC18327040093060004130A0500C1
:1073A00013871700179601002322E61EB387FA0001
:1073B000130650022380C700E312D7AE172703003D
:1073C00013074744B70610F0130717008347F7FF6A
:1073D00023A0F6F0832704009387F7FF1796010098
:1073E0002326F61AE39207FE130A05006FF01FAB7F
:1073F0001727030013070741130717008347F7FFF9
:107400002320F6F0832704009387F7FF9795010068
:1074100023AEF516E39207FE9386C6FF6FF09FC674
:10742000172703001307073EE39805FC9386C6FF62
:107430006FF05FC5E3FA9DBB930910006FF01FBFAB
:10744000130C000003C70C0093050700E30C07E4CE
:107450009308F0FF1305A00013080004B70610F00E
:10746000635E0B0C8327040013861700B387FA00B2
:1074700017930100232CC3102380E7006382A50823
:107480006308060B938C1C0003C70C00130CFCFF55
:1074900093050700E31607FCE35680E18327040009
:1074A0009305000213060004B70610F06F00C00039
:1074B000130CFCFFE3080CDE13871700B387FA00F8
:1074C0002380B700179501002322E50C93070700DE
:1074D000E310C7FE172703001307C732130717006F
:1074E0008347F7FF23A0F6F0832704009387F7FF75
:1074F00017950100232CF508E39207FE6FF05FFB60
:107500001727030013070730E30E06F613071700CB
:107510008347F7FF23A0F6F0832704009387F7FF44
:10752000179601002324F606E39207FE6FF09FF5FD
:10753000172703001307072D6FF05FFD130BFBFFE9
:10754000E3121BF36FF05FF5172703001307872B78
:10755000B70610F0130717008347F7FF23A0F6F0D4
:10756000832704009387F7FF179601002320F60274
:10757000E39207FE232421016FF05F92979C0100A4
:10758000938C4CE493050B0013850C00EF000077FF
:10759000330CAC40E35880EB83270400130600044F
:1075A000B70610F06F00C000130CFCFFE30A0CE8F4
:1075B00013871700B387FA0023807701979501009E
:1075C00023A6E5FC93070700E310C7FE1727030077
:1075D00013074723130717008347F7FF23A0F6F08D
:1075E000832704009387F7FF9795010023A0F5FAFE
:1075F000E39207FE6FF05FFB172703001307872056
:10760000E39806F4232421016FF05F89832781002A
:107610001387470083A707002324E10013DBF7410A
:107620006FF01FCB172703001307C71DB70610F015
:10763000130717008347F7FF23A0F6F08327040002
:107640009387F7FF179601002322F6F4E39207FED3
:107650009307100017970100232AF7F2930780077A
:10766000172703002300F71A6FF09FAF63568001BE
:107670009307D002E394FBF0979C0100938C8CD489
:1076800013078002930580026FF09FDC97260300AA
:1076900093864617370610F09386160003C7F6FF49
:1076A0002320E6F0032704001307F7FF9795010056
:1076B00023AEE5ECE31207FE6FF01FC4938D0700C5
:1076C000930CA000130D00006FF05F90B70710F04F
:1076D00023A0A7F26F000000130101FC1303410275
:1076E0002322B10293050300232E11002324C1029B
:1076F0002326D1022328E102232AF102232C0103AD
:10770000232E110323266100EFF00FF38320C10124
:10771000130500001301010467800000130101FB41
:1077200013038103232481022326A100232CC102F9
:1077300013040500130603001305C10023261102DC
:107740002322F104232ED1022320E1042324010566
:1077500023261105232E6100EFF04F9B8327C100E4
:10776000238007000325C1008320C1023305854023
:10777000032481021301010567800000B70710F0A0
:1077800083A647F403A607F403A747F4E31AD7FE3A
:10779000B7160000938606FAB306D60033B6C600C5
:1077A000B305E60023A4D7F423A6B7F4678000004E
:1077B000B70710F003A747F403A607F483A647F41E
:1077C000E31AD7FEB7160000938606FAB306D60072
:1077D00033B6C60023A4D7F4B305E60023A6B7F456
:1077E0009307000873A0473067800000130101FF72
:1077F000232481002326110097970100938787D9BE
:10780000179401001304C4D803A7070083270400BA
:107810001306F07C93064706938747069795010069
:1078200023AAD5D69795010023A4F5D6634AD6009E
:107830008320C1000324810013010101678000003F
:10784000130747899797010023A6E7D4EF00C049A3
:10785000930710006316F50203270400B717000012
:107860009387F77613050000E3D4E7FCEFF01FE6FB
:10787000032481008320C100130101016FB05FB7B1
:1078800017950100130585B4EFF01FE513052000DF
:10789000EFF0DFE3032481008320C1001301010125
:1078A0006FB01FB5179501001305C5B36FF0DFE288
:1078B00017950100130585B36FF01FE2130101FF57
:1078C000232481002322910023261100B7140000F5
:1078D00017940100130404B2938784381300000046
:1078E0009387F7FFE39C07FE13050400EFF0DFDE4C
:1078F0006FF09FFE6F008022130101FF232611000D
:10790000EF00803E1307100093070000631AE500A4
:107910008320C10013850700130101016780000067
:1079200017950100130585AAEFF01FDB8320C10026
:1079300093072000138507001301010167800000F1
:10794000737004306F0000006780000073700430B3
:107950006F000000130101FE232A9100232E110065
:10796000232C81002328210123263101835745033D
:107970001307901D930405006382E70E636EF70AF8
:107980006384070C1307801D639AE708139425008E
:1079900097290300938909EB33898900032509019D
:1079A0001306000093050900EFA04FEF9307B0FF07
:1079B0006304F514930710006306F50017970100A0
:1079C0002320F7BEB387890003A507021306000032
:1079D00093050900EFA00FDA9307C0FF6306F50ACD
:1079E0009307B0FF6308F50E930710006306F500D8
:1079F000179701002326F7BAB387890003A507016B
:107A00001306F0FF93050900EFA04FE99307C0FFAD
:107A1000E31EF5F89307801D239AF4028320C10129
:107A20000324810183244101032901018329C10029
:107A300013010102678000001307E01E6388E70658
:107A40001307F01EE39CE7FC97290300938989DF65
:107A500013942500338989006FF01FFA13942500D1
:107A600097290300938909DEB387890003A50702DC
:107A7000338989001306000093050900EFA08FCF1A
:107A80009307C0FFE31EF5F49307E01E239AF40268
:107A90008320C101032481018324410103290101C1
:107AA0008329C1001301010267800000139425009F
:107AB00097290300938909D933898900032509028D
:107AC0001306000093050900EFA0CFCA9307B0FF8B
:107AD000E31CF5F09307F01E239AF4028320C10102
:107AE0000324810183244101032901018329C10069
:107AF00013010102678000009307901D239AF4028E
:107B00008320C10103248101832441010329010150
:107B10008329C1001301010267800000130101FDE8
:107B2000232481022322910223202103232E3101C9
:107B3000232611022326010097240300938484D274
:107B400017290300130909D1130400009709000045
:107B5000938989E013060000930540001305100087
:107B6000EF900FC123A0A40013060000930540006E
:107B700013051000EF90CFBF2320A90003A5040038
:107B8000930600009305C10013060000EF908FD20A
:107B9000130604009305100013850900EF801FB938
:107BA0001304140093074000938444001309490010
:107BB000E312F4FA8320C1020324810283244102E8
:107BC000032901028329C101130101036780000019
:107BD000979701009387879C83A707001307301F9F
:107BE00093871700637CF70E130101FD2320210307
:107BF00017290300130909C72324810223229102B4
:107C0000232E3101232C41012326110297970100D5
:107C100023A607981304090097290300938989C5AF
:107C2000179A0100130A4A979304100003250400D1
:107C30001306C1009305810023260100EFA00FDE8B
:107C4000630E95069797010023AC979413044400A4
:107C5000E31E34FD83270A0017240300130484BFA6
:107C6000979901009389499393871700179701000B
:107C70002324F79293041000032504001306000048
:107C800093850900EFA0CFCE13044400630695004E
:107C90009797010023A69790E31089FE8320C102E5
:107CA0000324810283244102032901028329C101A3
:107CB000032A81011301010367800000032781006B
:107CC00083270A006306F7009797010023AA978C81
:107CD0008327C100E39807F66FF05FF7179701005D
:107CE000232EF78A67800000979701009387478BC0
:107CF00003A507001335150067800000B305B50024
:107D0000930705006386B70003C7070063160700E3
:107D10003385A74067800000938717006FF09FFEB0
:107D2000130101FB23229104232C410323229103FD
:107D3000232611042324810423202105232E31032B
:107D4000232A51032328610323267103232481035B
:107D50002320A103232EB101930C0500138A0500F3
:107D60009304000063DE05003305A0403337A00014
:107D7000B305B040930C0500338AE5409304F0FF4F
:107D800063DA06003306C040B337C000B306D04004
:107D9000B386F640930A06009389060013840C000C
:107DA00013090A0063960628178B0100130B8B50EA
:107DB0006370CA16B70701006372F6149307F00FD9
:107DC00063F4C70093098000B3573601330BFB00FF
:107DD00083470B0013050002B3873701B309F54051
:107DE000638C0900B3153A01B3D7FC00B31A36010E
:107DF00033E9B70033943C0113DB0A0193050B0010
:107E000013050900EF00507C130A050093050B00D1
:107E1000939B0A0113050900EF00907693DB0B0199
:107E20009305050013850B00EF00D072131A0A01A9
:107E300093570401B367FA0063FAA700B3875701A9
:107E400063E6570163F4A700B38757013389A7405E
:107E500093050B0013050900EF001077130A0500C6
:107E600093050B0013050900EF0090711314040132
:107E700093050500131A0A0113850B00135404011E
:107E8000EF00506D33648A00637AA4003304540118
:107E9000636654016374A400330454013304A440A2
:107EA0003354340193050000638A04003304804096
:107EB000B3378000B305B040B385F5401305040027
:107EC0008320C10403248104832441040329010481
:107ED0008329C103032A8103832A4103032B01035E
:107EE000832BC102032C8102832C4102032D01024A
:107EF000832DC1011301010567800000B707000150
:107F000093090001E362F6EC930980016FF0DFEB67
:107F1000631A06009305000013051000EF00506679
:107F2000930A0500B707010063FAFA0E9307F00FF2
:107F300063F4570193098000B3D73A01330BFB0078
:107F400083470B001305000233095A41B3873701F9
:107F5000B309F540E38209EAB39A3A01335BFA00C8
:107F6000B3153A01B3D7FC0093DB0A0133E9B7003C
:107F700013050B0093850B00EF001065130A050035
:107F800093850B00139C0A0113050B00EF00505F53
:107F9000135C0C019305050013050C00EF00905BCA
:107FA000131A0A0193570901B367FA0033943C018D
:107FB00063FAA700B387570163E6570163F4A7008C
:107FC000B3875701338BA74093850B0013050B0034
:107FD000EF00905F130A050093850B0013050B005B
:107FE000EF00105A9305050013050C00EF009056A2
:107FF00093160901131A0A0193D60601B366DA0033
:1080000063FAA600B386560163E6560163F4A60040
:10801000B38656013389A6406FF01FDEB707000113
:1080200093090001E3EAFAF0930980016FF0DFF0B1
:108030006376DA0093050A006FF01FE7B7070100C7
:1080400063FAF604930BF00F33B5DB00131535001C
:1080500033D7A600978701009387C725B387E7002A
:1080600083CB070093050002B38BAB00338B7541C4
:10807000631C0B0263E4460163EACC003384CC400A
:10808000B306DA4033B98C003389264193050900E1
:108090006FF09FE1B707000113050001E3EAF6FA6C
:1080A000130580016FF0DFFAB3966601335D760148
:1080B000336DDD00B35D7A01B3156A0133DC7C01F9
:1080C00013540D01336CBC0013850D00930504009F
:1080D000B3196601EF00504F930A050093050400A1
:1080E00013850D0033996C01931C0D01EF0050496D
:1080F00093DC0C01130A05009305050013850C00A1
:10810000EF005045939A0A0113570C0133E7EA0038
:10811000930D0A00637EA7003307A701930DFAFFB2
:108120006368A7016376A700930DEAFF3307A701F1
:10813000330AA7409305040013050A00EF00D04856
:1081400093050400930A050013050A00EF0050434D
:10815000930505001304050013850C00EF00903F04
:1081600093150C01939A0A0193D50501B3E5BA0062
:108170001307040063FEA500B385A5011307F4FFF0
:1081800063E8A50163F6A5001307E4FFB385A50125
:10819000939D0D01B70C0100B3EDED001384FCFFBE
:1081A000B3F78D0033F48900338AA54013850700A7
:1081B000930504002326F10093DD0D01EF009039B3
:1081C00093050400930A050013850D00EF00903815
:1081D00013DC090193050C002324A10013850D0075
:1081E000EF0050378327C10013040C0093050400EF
:1081F000130C050013850700EF00D035832681009E
:1082000013D70A013305D5003307A7006374D700DD
:10821000330C9C01B70701009387F7FF93550701C3
:108220003377F70013170701B3F7FA00B385850119
:10823000B307F7006366BA00631EBA00637CF900F7
:1082400033863741B3B7C700B385A541B385F54041
:1082500093070600B307F9403339F900B305BA4074
:10826000B385254133947501B3D767013364F400B6
:10827000B3D565016FF05FC3130101FD23229102A5
:10828000232A5101232611022324810223202103C2
:10829000232E3101232C4101232861012326710162
:1082A00023248101232291012320A101930A0500A7
:1082B00093840500639E06381304060093090500A5
:1082C00017890100130909FF63F8C512B7070100F8
:1082D000138B05006378F6101307F00F3337C700D0
:1082E00013173700B357E6003309F9008346090036
:1082F0003387E60093060002B386E640638C0600EF
:10830000B394D40033D7EA003314D600336B97000C
:10831000B399DA00935A040193850A0013050B0000
:10832000EF00902A1309050093850A00931B0401AE
:1083300013050B00EF00D02493DB0B019304050021
:108340009305050013850B00EF00D02013190901D8
:1083500093D70901B367F900138A040063FEA700ED
:10836000B3878700138AF4FF63E8870063F6A700EA
:10837000138AE4FFB3878700B384A74093850A007C
:1083800013850400EF0050241309050093850A00AB
:1083900013850400EF00D01E939909019304050092
:1083A000930505001319090113850B0093D90901E1
:1083B000EF00501AB36939011386040063FCA90069
:1083C000B30934011386F4FF63E6890063F4A9005E
:1083D0001386E4FF13140A013364C400130A000077
:1083E0006F000013B707000113070001E36CF6EEFE
:1083F000130780016FF01FEF138A0600631A06004F
:108400009305000013051000EF00901713040500FA
:10841000B7070100637EF4129307F00F63F487003F
:10842000130A8000B35744013309F90003470900D8
:108430009306000233074701B386E64063940612B1
:10844000B3848440130A1000135B040193050B00EE
:1084500013850400EF0050171309050093050B0066
:1084600013850400931B0401EF00901193DB0B01B3
:10847000930405009305050013850B00EF00900D94
:108480001319090193D70901B367F900938A04000E
:1084900063FEA700B3878700938AF4FF63E8870031
:1084A00063F6A700938AE4FFB3878700B384A740ED
:1084B00093050B0013850400EF001011130905004C
:1084C00093050B0013850400EF00900B93990901AD
:1084D00093040500930505001319090113850B008A
:1084E00093D90901EF001007B3693901138604001D
:1084F00063FCA900B30934011386F4FF63E6890025
:1085000063F4A9001386E4FF13940A013364C400E2
:108510001305040093050A008320C102032481028D
:1085200083244102032901028329C101032A810115
:10853000832A4101032B0101832BC100032C8100FD
:10854000832C4100032D010013010103678000000B
:10855000B7070001130A0001E366F4EC130A800177
:108560006FF05FEC3314D40033DAE400B399DA002F
:1085700033D7EA00935A0401B394D40093850A00D8
:1085800013050A00336B9700EF0010041309050070
:1085900093850A0013050A00931B0401EF00407E37
:1085A00093DB0B01930405009305050013850B0075
:1085B000EF00407A1319090113570B013367E900E3
:1085C000138A0400637EA70033078700138AF4FF31
:1085D000636887006376A700138AE4FF3307870088
:1085E000B304A74093850A0013850400EF00C07D03
:1085F0001309050093850A0013850400EF004078F5
:10860000930405009305050013850B00EF008074AB
:1086100013170B011357070113190901B367E90079
:108620001387040063FEA700B38787001387F4FF56
:1086300063E8870063F6A7001387E4FFB38787002A
:10864000131A0A01B384A740336AEA006FF0DFDF30
:1086500063ECD51EB707010063F4F6041307F00FAF
:10866000B335D7009395350033D7B600978701000F
:10867000938747C4B387E70003C70700130A0002C4
:108680003307B700330AEA4063160A0213041000E6
:10869000E3E096E833B6CA00134416006FF05FE7D4
:1086A000B707000193050001E3E0F6FC93058001A4
:1086B0006FF09FFBB35CE600B3964601B3ECDC00C1
:1086C00033D4E40093DB0C01B397440133D7EA00C1
:1086D00093850B0013050400336BF700B3194601B3
:1086E000EF00806E1309050093850B00130504004D
:1086F000139C0C01EF00C068135C0C01930405008F
:108700009305050013050C00EF00C064131909015F
:1087100013570B013367E90013840400637EA7003D
:10872000330797011384F4FF636897016376A7000A
:108730001384E4FF33079701B304A74093850B002C
:1087400013850400EF0040681309050093850B00B2
:1087500013850400EF00C062930405009305050033
:1087600013050C00EF00005F93170B0113190901AB
:1087700093D70701B367F9001386040063FEA700CF
:10878000B38797011386F4FF63E8970163F6A700A8
:108790001386E4FFB387970113140401B70B01009C
:1087A0003364C4001389FBFF337D240133F92901AD
:1087B000B384A7409305090013050D00EF0080590D
:1087C000935C040193050900130B050013850C004D
:1087D000EF00405893D90901130C05009385090057
:1087E00013850C00EF00005713090500938509005D
:1087F00013050D00EF0000563305850193570B015B
:108800003385A70063748501330979019357050106
:10881000B387270163E6F402E392F4BCB7070100D3
:108820009387F7FF3375F50013150501337BFB00C4
:1088300033964A0133056501130A0000E37AA6CC9A
:108840001304F4FF6FF09FB9130A00001304000033
:108850006FF01FCC130101FB232481042322910418
:10886000232E3103232291032326110423202105E3
:10887000232C4103232A5103232861032326710358
:10888000232481032320A103232EB101930C05008F
:10889000938905001304050093840500639E062652
:1088A00013090600138A0600978A0100938A8AA09A
:1088B00063F4C514B70701006376F6129307F00F4F
:1088C00063F4C700130A8000B3574601B38AFA0065
:1088D00003C70A001305000233074701330AE540C6
:1088E000630C0A00B395490133D7EC0033194601F4
:1088F000B364B70033944C01935A090193850A007D
:1089000013850400EF00404C9309050093850A008D
:10891000131B090113850400EF008046135B0B0154
:108920009305050013050B00EF00C0429399090160
:1089300093570401B3E7F90063FAA700B38727014F
:1089400063E6270163F4A700B3872701B384A74038
:1089500093850A0013850400EF0000479309050082
:1089600093850A0013850400EF008041131404016D
:10897000930505009399090113050B001354040195
:10898000EF00403D33E48900637AA40033042401FE
:10899000636624016374A400330424013304A440F7
:1089A00033554401930500008320C104032481044E
:1089B00083244104032901048329C103032A810379
:1089C000832A4103032B0103832BC102032C810261
:1089D000832C4102032D0102832DC10113010105E6
:1089E00067800000B7070001130A0001E36EF6EC90
:1089F000130A80016FF05FED631A06009305000013
:108A000013051000EF00C03713090500B707010078
:108A1000637AF90E9307F00F63F42701130A8000BD
:108A2000B3574901B38AFA0003C70A0013050002CD
:108A3000B384294133074701330AE540E30E0AEACC
:108A400033194901B3DAE900B395490133D7EC0092
:108A500093540901336BB70013850A009385040012
:108A6000EF0080369309050093850400931B0901EC
:108A700013850A00EF00C03093DB0B01930505005E
:108A800013850B00EF00002D9399090193570B01FB
:108A9000B3E7F90033944C0163FAA700B3872701C9
:108AA00063E6270163F4A700B3872701B38AA740D1
:108AB0009385040013850A00EF0000319309050037
:108AC0009385040013850A00EF00802B93050500B1
:108AD00013850B00EF00002893150B0193990901F2
:108AE00093D50501B3E5B90063FAA500B385250167
:108AF00063E6250163F4A500B3852501B384A54091
:108B00006FF09FDFB7070001130A0001E36AF9F075
:108B1000130A80016FF0DFF0E3E8D5E8B707010042
:108B200063FCF604930BF00F33B5DB00131535002F
:108B300033D7A600977701009387C777B387E700FD
:108B400083CB070093050002B38BAB00338B7541D9
:108B5000631E0B0263E4360163EACC003384CC402D
:108B6000B386D94033B58C00B384A6401305040006
:108B7000938504006FF05FE3B70700011305000160
:108B8000E3E8F6FA130580016FF09FFAB3966601E9
:108B9000335D7601336DDD0033D47901B39569011E
:108BA00033DC7C0193540D01336CBC0013050400CD
:108BB00093850400B31A6601EF000021130A050033
:108BC000938504001305040033996C01931C0D0177
:108BD000EF00001B93DC0C01130405009305050056
:108BE00013850C00EF000017131A0A0113570C012C
:108BF0003367EA00130A0400637EA7003307A70166
:108C0000130AF4FF6368A7016376A700130AE4FF61
:108C10003307A701B309A740938504001385090012
:108C2000EF00801A938504001304050013850900E2
:108C3000EF000015930505009304050013850C0053
:108C4000EF00401193150C011314040193D5050195
:108C5000B365B4001387040063FEA500B385A501C6
:108C60001387F4FF63E8A50163F6A5001387E4FF0B
:108C7000B385A501131A0A01B70C0100336AEA0093
:108C80001384FCFFB3778A0033F48A00B384A540D1
:108C900013850700930504002326F100135A0A01E7
:108CA000EF00400B930905009305040013050A002B
:108CB000EF00400A13DC0A01930D050093050C0038
:108CC00013050A00EF0000098327C100130A0500FD
:108CD00093050C0013850700EF00C0073305B501AD
:108CE00013D709013307A7006374B701330A9A0148
:108CF000B70701009387F7FF935507013377F70014
:108D000013170701B3F7F900B3854501B307F7005F
:108D100063E6B400639EB400637CF9003386574178
:108D2000B3B7C700B385A541B385F54093070600E7
:108D3000B307F9403339F900B385B440B385254111
:108D400033947501B3D767013365F400B3D565017A
:108D50006FF09FC5130605001305000093F615007C
:108D6000638406003305C50093D51500131616005D
:108D7000E39605FE678000006340050663C60506AE
:108D800013860500930505001305F0FF630C06022A
:108D900093061000637AB6006358C00013161600DD
:108DA00093961600E36AB6FE1305000063E6C5005D
:108DB000B385C5403365D50093D61600135616000B
:108DC000E39606FE6780000093820000EFF05FFBF1
:108DD00013850500678002003305A04063D80500B5
:108DE000B305B0406FF0DFF9B305B04093820000E7
:108DF000EFF01FF93305A040678002009382000066
:108E000063CA0500634C0500EFF09FF7138505006A
:108E100067800200B305B040E35805FE3305A0406B
:108E2000EFF01FF63305B04067800200977701002E
:108E30009387477383A607001777010013074771CD
:108E40000327070023A2A600637EE5001777010031
:108E50001307C7700325070083A507009385450006
:108E60006F70DFE8130101FF232481002326110026
:108E7000177701001307C76E1304050003250700C9
:108E800083A5070093854500EF705FE697770100A3
:108E90009387476A83A707006376F40097770100FA
:108EA00023AA87688320C1000324810013010101E4
:108EB00067800000977701009387C76A03A70700C0
:108EC00083A60700832747049387F7FF2322F7042D
:108ED00083A7460463940700736004306780000032
:108EE000130101FE232C8100232A910013040500A5
:108EF00093840500232821012326310123244101E5
:108F000023225101232E1100EFA08FCF83270400CD
:108F100003290401B7090001B3E59700930AC400CF
:108F20002320B400930400009389F9FF370A00025C
:108F30000327040063822A0503260900130509009C
:108F4000B3654701B37636019317560033F7E60051
:108F50000329490063C60700631607006FF05FFD31
:108F6000E398E6FC9317760063D40700B3E4D400DB
:108F7000EFB05F916FF0DFFB93C4F4FFB3F4E40054
:108F800023209400EFA04FFB032504008320C101A0
:108F90000324810183244101032901018329C100A4
:108FA000032A8100832A4100130101026780000027
:108FB000130101FF2326110023248100EFE01FB6D7
:108FC00017F7FFFF1307C782930600001306100070
:108FD000930540061775010013054542EFC0DFC039
:108FE0006302050213040500EFA00FC3130605007A
:108FF00013070000930600009305100013050400FA
:10900000EFC09FD0EFA00F8D8320C100032481000B
:0C9010001305000013010101678000003F
:02000004800278
:10000000046CFEFF746DFEFF106CFEFF746DFEFF4E
:10001000746DFEFF746DFEFF746DFEFF386CFEFFA5
:10002000746DFEFF746DFEFF606CFEFF706CFEFF72
:10003000746DFEFF886CFEFF986CFEFF986CFEFFEF
:10004000986CFEFF986CFEFF986CFEFF986CFEFFAC
:10005000986CFEFF986CFEFF986CFEFF746DFEFFBF
:10006000746DFEFF746DFEFF746DFEFF746DFEFF18
:10007000746DFEFF746DFEFF746DFEFF746DFEFF08
:10008000746DFEFF746DFEFF746DFEFF746DFEFFF8
:10009000746DFEFF746DFEFF746DFEFF746DFEFFE8
:1000A000746DFEFF746DFEFF746DFEFF746DFEFFD8
:1000B000746DFEFF746DFEFF746DFEFF746DFEFFC8
:1000C000746DFEFF746DFEFF746DFEFF746DFEFFB8
:1000D000746DFEFF746DFEFF746DFEFF746DFEFFA8
:1000E000746DFEFF746DFEFF746DFEFF746DFEFF98
:1000F000746DFEFF746DFEFF746DFEFF746DFEFF88
:10010000DC6CFEFF046DFEFF746DFEFF746DFEFF80
:10011000746DFEFF746DFEFF746DFEFF746DFEFF67
:10012000746DFEFF646DFEFF746DFEFF746DFEFF67
:10013000146AFEFF1C6BFEFF746DFEFF746DFEFF04
:100140006C6BFEFF746DFEFFE46BFEFF746DFEFFD3
:10015000746DFEFF2C6CFEFFD071FEFF3C72FEFF43
:10016000DC71FEFF3C72FEFF3C72FEFF3C72FEFF44
:100170003C72FEFF7470FEFF3C72FEFF3C72FEFF9D
:100180009C70FEFFAC70FEFF3C72FEFFC470FEFF71
:10019000D470FEFFD470FEFFD470FEFFD470FEFF5B
:1001A000D470FEFFD470FEFFD470FEFFD470FEFF4B
:1001B000D470FEFF3C72FEFF3C72FEFF3C72FEFFFD
:1001C0003C72FEFF3C72FEFF3C72FEFF3C72FEFF83
:1001D0003C72FEFF3C72FEFF3C72FEFF3C72FEFF73
:1001E0003C72FEFF3C72FEFF3C72FEFF3C72FEFF63
:1001F0003C72FEFF3C72FEFF3C72FEFF3C72FEFF53
:100200003C72FEFF3C72FEFF3C72FEFF3C72FEFF42
:100210003C72FEFF3C72FEFF3C72FEFF3C72FEFF32
:100220003C72FEFF3C72FEFF3C72FEFF3C72FEFF22
:100230003C72FEFF3C72FEFF3C72FEFF3C72FEFF12
:100240003C72FEFF3C72FEFF3C72FEFF3C72FEFF02
:100250003C72FEFF3C72FEFF1871FEFF5471FEFF00
:100260003C72FEFF3C72FEFF3C72FEFF3C72FEFFE2
:100270003C72FEFF3C72FEFF3C72FEFFC071FEFF4F
:100280003C72FEFF3C72FEFF486EFEFF9C6FFEFF5D
:100290003C72FEFF3C72FEFF2C70FEFF3C72FEFFC4
:1002A0005870FEFF3C72FEFF3C72FEFF3072FEFF94
:1002B000000102020303030304040404040404040D
:1002C00005050505050505050505050505050505DE
:1002D00006060606060606060606060606060606BE
:1002E00006060606060606060606060606060606AE
:1002F000070707070707070707070707070707078E
:10030000070707070707070707070707070707077D
:10031000070707070707070707070707070707076D
:10032000070707070707070707070707070707075D
:10033000080808080808080808080808080808083D
:10034000080808080808080808080808080808082D
:10035000080808080808080808080808080808081D
:10036000080808080808080808080808080808080D
:1003700008080808080808080808080808080808FD
:1003800008080808080808080808080808080808ED
:1003900008080808080808080808080808080808DD
:1003A00008080808080808080808080808080808CD
:1003B000546D725100000000546D7220537663003A
:1003C000286E756C6C2900004572726F7220696E20
:1003D00020787878207461736B73200D0A00000018
:1003E0006D69616F750A00006D69616F75320A0091
:1003F00068756E6772790A00436865636B54696D4E
:040400006572000021
:100404001000000000000000017A5200017C01018C
:100414001B0D020050000000180000000079FEFFD0
:100424005805000000440E507489039406990B810A
:1004340001880292049305950796089709980A9AE9
:100444000C9B0D036C010AC144C844C944D244D373
:1004540044D444D544D644D744D844D944DA44DBBC
:10046400440E00440B0000004C0000006C0000002F
:10047400047EFEFFDC05000000440E307089039505
:1004840007810188029204930594069608970998B7
:100494000A990B9A0C0370020AC144C844C944D295
:1004A40044D344D444D544D644D744D844D944DA74
:1004B400440E00440B00000050000000BC0000008B
:1004C4009083FEFF0005000000440E5074880289EA
:1004D400039305990B810192049406950796089756
:1004E40009980A9A0C9B0D0320010AC144C844C907
:1004F40044D244D344D444D544D644D744D844D92C
:0C05040044DA44DB440E00440B0000000D
:0805A000FC8F010009000000BE
:040000058000004037
:00000001FF
